:020000020000FC
:100000000C941C140C943D0F0C94700F0C94001461
:100010000C94060E0C94090E0C94070E0C94080E0A
:100020000C94F30D0C94F40D0C94F50D0C94F60D4A
:100030000C94F70D0C94F80D0C94F90D0C94FA0D2A
:100040000C94FB0D0C94FC0D0C94A30F0C94000E5F
:100050000C94D5120C941A130C94010E0C94FE0DF2
:100060000C943D130C94FD0D0C94FF0D0C94050E97
:100070000C94020E0C94030E0C94040E8954400B45
:10008000B83630303000895A1C05783238303000AC
:10009000895A1C04B03234303000895A1C041A3298
:1000A00031303000895A1C03843138303000895790
:1000B0002E01F4313030300089572E00C820343002
:1000C000300089572E007D20323530008954400B96
:1000D000B836303030001F2864110001B0001D0018
:1000E000B8000D001F2864110001B8000D00E000E9
:1000F0000D001F2864110001E0000D00E8001D0044
:100100001F2864110001BB001D00C3000D001F2843
:1001100064110001C3000D00D5000D001F286411FB
:100120000001D5000D00DD001D001F286411000135
:10013000BC001D00C4000D001F2864110001C40094
:100140000D00D4000D001F2864110001D4000D0023
:10015000DC001D001F2864110001BD001D00C5004A
:100160000D001F2864110001C5000D00D3000D0013
:100170001F2864110001D3000D00DB001D001F28A3
:1001800064110001BE001D00C6000D001F2864118F
:100190000001C6000D00D2000D001F2864110001EF
:1001A000D2000D00DA001D001F2864110001C000FC
:1001B0001D00C8000D001F2864110001C8000D00BB
:1001C000D0000D001F2864110001D0000D00D800E0
:1001D0001D001F2864110001C2001D00CA000D008F
:1001E0001F2864110001CA000D00CE000D001F2859
:1001F00064110001CE000D00D6001D001F286411FF
:100200000001C4001D00CB000D001F286411000177
:10021000CB000D00CD000D001F2864110001CD00A2
:100220000D00D5001D001F2864110001B0000D0055
:10023000B8001D001F2864110001B8001D00E00077
:100240001D001F2864110001E0001D00E8000D00E2
:1002500006F15827102032304B0006F1580B543568
:100260003830300006F1580578323830300006F169
:10027000580514323630300006F158041A32313045
:10028000300006F15803E8323030300006F15803F0
:1002900084313830300006F15801F431303030000C
:1002A00006F15800FA203530300006F15800C82019
:1002B0003430300006F1580096203330300006F11B
:1002C00058007D203235300006F158003E20313292
:1002D000350006F15827102032304B001F286411DA
:1002E0000001B0001D00B70010001F2864110001BC
:1002F000B7001000E10010001F2864110001E100A8
:100300001000E8001D001F2864110001B2001D004C
:10031000B90010001F2864110001B9001000DF00AF
:1003200010001F2864110001DF001000E6001D000E
:100330001F2864110001BC001D00C30010001F280D
:1003400064110001C3001000D50010001F286411C3
:100350000001D5001000DC001D001F286411000101
:10036000BD001D00C40010001F2864110001C4005E
:100370001000D40010001F2864110001D4001000E8
:10038000DB001D001F2864110001BE001D00C50018
:1003900010001F2864110001C5001000D3001000D8
:1003A0001F2864110001D3001000DA001D001F286F
:1003B00064110001BF001D00C60010001F28641159
:1003C0000001C6001000D20010001F2864110001B7
:1003D000D2001000D9001D001F2864110001C000C8
:1003E0001D00C70010001F2864110001C700100085
:1003F000D10010001F2864110001D1001000D800A6
:100400001D001F2864110001C1001D00C80010005C
:100410001F2864110001C8001000D00010001F2820
:1004200064110001D0001000D7001D001F286411C6
:100430000001C2001D00C90010001F286411000146
:10044000C9001000CF0010001F2864110001CF0068
:100450001000D6001D001F2864110001C3001D00FC
:10046000CA0010001F2864110001CA001000CE004D
:1004700010001F2864110001CE001000D5001D00DF
:100480001F2864110001C4001D00CB0010001F28AC
:1004900064110001CB001000CD0010001F28641172
:1004A0000001CD001000D4001D001F2864110001C0
:1004B000C5001D00CC0010001F2864110001CC00F5
:1004C0001000CC0010001F2864110001CC001000A7
:1004D000D3001D001F2864110001C6001D00CD00BF
:1004E00010001F2864110001CD001000CB00100087
:1004F0001F2864110001CB001000D2001D001F282E
:1005000064110001B0000D00B7001D001F28641128
:100510000001B7001D00E1001D001F28641100014B
:10052000E1001D00E8000D001F2864110001CC004F
:100530002000CC000A001F286411020098000A0065
:10054000FF001D001F24BE0000001F2867010120BE
:10055000504120566F6C74732D3E20524620436FDD
:100560006D702D3E2020202020414C432D3E202028
:100570002020205357522D3E20467764205077721A
:100580002D3E5265666C205077722D3E20504120E2
:10059000437572722D3E44767220437572722D3E01
:1005A0000C1F286701011F24780002001F28670123
:1005B000026B487A1F5800FF1F5811FF1F5812FF87
:1005C0001F5813FF1F5814FF1F5815FF1F5816FF01
:1005D0001F5817FF1F5818FF0B1F28670104000042
:1005E0000000001F286701020A2E000000FF0B1FF9
:1005F000286701042020202020000B1F2867010409
:100600000000001F286701021F24380002000000BC
:10061000002E000000FF1F24000004001F286701B7
:10062000015478204F6E1F24880001001F286701A5
:10063000012E20FF1F286411020098000800FF000F
:100640002E001F24420005001F28670101523AFFB7
:1006500043572855534229204357284C53422920B9
:1006600055534220202020204C534220202020207F
:10067000414D202020202020464D202020202020D9
:100680004449472855534229444947284C53422955
:100690001F24000005001F28670101583AFF1F248E
:1006A000DA0007001F28670101502DFF1F24CC002E
:1006B00007001F286701015420FF1F248200050046
:1006C0001F28670101FF1F249A0004001F286701EB
:1006D000012A393A20202020202020343AFF1F24EC
:1006E000680004001F286701014C6F636BFF1F2423
:1006F000000002001F286701024F7574206F6620FA
:1007000062616E6421FF1F24000002001F28670140
:100710000252414D20746573742070617373656477
:100720006661696C65640C1F24000002001F286765
:10073000010250726F632073796E63206661696C89
:1007400065641F24920000001F28670101202020FB
:1007500020202061416242634364446545664667E8
:1007600047684869496A4A6B4B6C4C6D4D6E4E6FD9
:100770004F70507151725273537454755576567749
:1007800057785879597A5A303132333435363738C8
:10079000393F2C2E2F2D3D2B282623252A3A3B216D
:1007A000402924275F3C1F24000004001F28670104
:1007B00001202020202020202020202020FF0C1F8E
:1007C00024200002001F286701044143763A414774
:1007D000A23A4148BB3A414CD43A414EEF3A4150DB
:1007E000423B4152193B41545C3B42527C3B4341AA
:1007F000B33B4342AD3B4343D73B4344ED3B4346CE
:10080000903B434C143C434D253C434F743C435078
:10081000903C4352363C4353A13C4355033C435820
:10082000B23C4446CA3C444EC33C4454DB3C445571
:10083000F53C4456193D45532D3D4641503D4642F9
:100840005C3D4644683D4649873D464EAF3D465275
:10085000393E4653843E46545C3E4657A13E465878
:10086000313F4659593F47547D3F4853A63F49447D
:10087000BC3F4946C43F4952E23D4953464049586E
:10088000F43D4959043E4B4DAF404B53D0404B597A
:10089000F0404C431F414C4B38414C5453414D4266
:1008A0006C414D4385414D44AC414D47E1414D5272
:1008B000FA414D558B424D574C424E42AF424E5439
:1008C000CD424E57EA4250410F4350433C435044BF
:1008D0008043504CA043504DBD435052DC435053D5
:1008E0000044505419445057534451537144524199
:1008F00095445243C5445244CA445246F044524778
:100900000345524B2045524D484552509045525454
:1009100096455255D7445258BA455342CB45534356
:1009200002465344A0465345D14653491946534DB8
:10093000E84653503046535112475353514653548F
:1009400072465356894654432F4754464E47544C9B
:100950005F47544D7847545287475458EA4555509D
:10096000493D5641A4475644BD475647EE47565861
:1009700000485843564858445B48585432485855E4
:100980006848585681481F245800000008084357FB
:100990002855534229204357284C53422920555368
:1009A0004220202020204C53422020202020414D56
:1009B000202020202020464D202020202020444997
:1009C000472855534229444947284C5342291F245C
:1009D0000000070000044147432D04044175746F73
:1009E00046617374536C6F774F6666201F243C001A
:1009F000070000034E422D02046F6666206F6E20D2
:100A000020FF1F246C00070005044D4F5820505450
:100A1000542050545443564F5820564F58431F2487
:100A20008A000700000352782D02015452FF1F2450
:100A3000AC000700000354782D02014142FF1F243F
:100A40009800010000074D657465723A20080A504D
:100A50004120566F6C74732020524620436F6D7096
:100A6000202020414C43202020202020205357527A
:100A700020202020202020467764205077722020DC
:100A8000205265666C2050777220205041204375BB
:100A9000727220202044767220437572722020FFEB
:100AA0001F2498000200000D4272696768746E6529
:100AB00073733A202008044C6F77304C6F77314CB9
:100AC0006F77324C6F77334D6564314D6564324DCD
:100AD00065643348696768FF1F24980003000007B6
:100AE00050205320423A20020A4F666620202020E0
:100AF0002020204F6E2020202020202020FF1F2497
:100B000098000400000F44697370207265732028F8
:100B1000487A293A20020231302031FF1F24980000
:100B20000500000D46756C6C204475706C65783A54
:100B30002002044F6666204F6E2020FF1F2498007D
:100B40000100000E5054542D524620286D73293A4E
:100B500020201E032020312020322020332020346A
:100B60002020352020362020372020382020392012
:100B700031302031312031322031332031342031B5
:100B8000352031362031372031382031392032308C
:100B9000203231203232203233203234203235209C
:100BA00032362032372032382032392033301F2479
:100BB00098000200000A504320417564696F3A2092
:100BC000020744697361626C65456E61626C652001
:100BD0001F2498000300000A547820417564696F4F
:100BE0003A2002074D6963202020204C696E652061
:100BF00020201F2498000400000C4C6F636B2074AD
:100C0000696D65723A2004054F66662020313073A5
:100C10002020333073202036307320201F2498008A
:100C20000500000C506F77657220736176653A207D
:100C300004054F6666202031356D696E33306D696D
:100C40006E36306D696E1F2498000100000C5069EB
:100C50007463682028487A293A2001F81F249800F4
:100C60000200000D5370656564202877706D293A85
:100C70002001F8FF1F2498000300000E456E6861F4
:100C80006E636564205353423A2002034F66662028
:100C90004F6E1F2498000400000E464D20446576D8
:100CA00020286B487A293A200303322E30342E3024
:100CB000352E30FF1F2498000500000F4C69636536
:100CC0006E736520636C6173733A200502452041A1
:100CD00020472054204E20FF1F24980001000009C7
:100CE000565041202856293A2001FAFF1F24980027
:100CF00002000009495041202841293A2001FAFF09
:100D00001F24980003000009494476202841293A0D
:100D10002001FAFF1F24980004000009436D702889
:100D20006442293A2001FAFF1F24980005000009B7
:100D3000414C43202856293A2001FAFF1F249800ED
:100D400001000009535752202020203A2001FAFFC9
:100D50001F24980002000009467764202857293A8A
:100D60002001FAFF1F249800030000095265662045
:100D70002857293A2001FAFF1F2498000400000A8E
:100D8000202020202020202020200207202020209A
:100D9000202020202020202020201F249800050033
:100DA000000A2020202020202020202002072020B0
:100DB0002020202020202020202020201F249800D8
:100DC0000100000E564F58206761696E3A202020BE
:100DD0002020FFF81F2498000200000E564F5820D4
:100DE00073656E733A2020202020FFF81F2498009E
:100DF0000300000E416E7469564F58206761696E9A
:100E00003A20FFF81F2498000400000E564F582087
:100E1000646C792831306D73293AFFF81F249800EB
:100E20000500000A4D696320426961733A20020798
:100E30004F6666202020203920566F6C74731F2463
:100E4000980001000005416D703A20040C4E6F6E51
:100E5000652020202020202020496E74203130572A
:100E60002020202020496E7420313030572020204F
:100E700020496E7420313030572B457874FF1F2481
:100E800098000200000C4B65796572204D6F646517
:100E90003A20030549616D624149616D6242556CBA
:100EA00074696DFF1F2498000300000E4661726E86
:100EB00073776F7274683A20202011034F666620A2
:100EC000203520203620203720203820203920319E
:100ED000302031312031322031332031342031354E
:100EE000203136203137203138203139203230FF5F
:100EF0001F2498000400000E53424920646C792896
:100F000031306D73293AFFF81F2498000500000E58
:100F100046424920646C79286D73293A2020FFF8F5
:100F20001F2498000100000E5876657274657220C7
:100F3000467265713A2017036F6666353020353288
:100F40002035342031343431343632323232323496
:100F5000343230343232343234343236343238345B
:100F60003330343332343334343336343338343446
:100F700030343432343434343436343438FF1F248B
:100F80009800020000094454523D5054543A200243
:100F9000084E6F202020202020596573202020201B
:100FA00020FF1F2498000300000B4261756420722B
:100FB0006174653A200506202039363030203139F9
:100FC000323030203338343030203537363030311D
:100FD0003135323030FF1F2498000400000A486188
:100FE0006E647368616B653A02072020204E6F6E55
:100FF000654354532F5254531F2498000500000D8D
:101000005475726E6F6E20646973703A200204200A
:101010004F66664D736731FF1F2498000100000B77
:101020005363616E20747269703A20050620202097
:1010300020533520202020533620202020533720D5
:101040002020205338202020205339FF1F249800CF
:101050000200000C5363616E2073746172743A2055
:10106000FFF81F2498000300000B5363616E207388
:10107000746F703A20FFF8FF1F2498000400000EE0
:101080004672657120696E6328487A293A200903FF
:1010900063686E20313031303020314B31304B318C
:1010A000354B32304B32354B35304BFF1F249800D7
:1010B0000500000D4477656C6C20286D73293A207B
:1010C00020050420313030203235302035303031A9
:1010D00030303035303030FF1F24980001000006DA
:1010E000526F6F663A20020B37302E3030304D4849
:1010F0007A202037302E3435354D487A20201F2471
:10110000980002000008394D487A2D313A20010933
:10111000363030302020202020FF1F24980003008C
:101120000008394D487A2D323A20090936303030DE
:10113000202020202032383030202020202032343F
:10114000303020202020203231303020202020203C
:101150003138303020202020203130303020202005
:101160002020343030202020202020323530202014
:10117000202020206E6F6E652020202020FF1F245D
:10118000980004000008394D487A2D333A200909A7
:1011900036303030202020202032383030202020BF
:1011A00020203234303020202020203231303020B6
:1011B00020202020313830302020202020313030B5
:1011C00030202020202034303020202020202032C9
:1011D00035302020202020206E6F6E6520202020BA
:1011E00020FF1F24980005000008394D487A2D344F
:1011F0003A20090936303030202020202032383083
:101200003020202020203234303020202020203276
:101210003130302020202020313830302020202054
:101220002031303030202020202034303020202049
:101230002020203235302020202020206E6F6E6547
:101240002020202020FF1F2498000100000A3435B0
:10125000354B487A2D313A20020732304B2020207E
:1012600020353830302020201F2498000200000A4A
:101270003435354B487A2D323A200E0732304B2028
:1012800020202035383030202020323830302020C7
:1012900020323630302020203231303020202032B1
:1012A0003030302020203138303020202031303094
:1012B00030202020353030202020203430302020B5
:1012C00020203330302020202032353020202020B4
:1012D000313235202020206E6F6E652020201F24A3
:1012E00098000300000A3435354B487A2D333A20F4
:1012F0000E0732304B20202020353830302020207F
:101300003238303020202032363030202020323128
:101310003030202020323030302020203138303022
:101320002020203130303020202035303020202047
:101330002034303020202020333030202020203234
:10134000353020202020313235202020206E6F6E55
:10135000652020201F2498000400000A3435354BF6
:10136000487A2D343A200E0732304B202020203589
:1013700038303020202032383030202020323630B3
:1013800030202020323130302020203230303020C8
:1013900020203138303020202031303030202020C3
:1013A00035303020202020343030202020203330B1
:1013B00030202020203235302020202031323520AE
:1013C0002020206E6F6E652020201F2498000500CD
:1013D000000A20202020202020202020020720207A
:1013E0002020202020202020202020201F249800A2
:1013F0000100000D5246472063616C202846293ABF
:1014000020FFF8FF1F2498000200000D52464720DD
:1014100063616C202853293A20FFF8FF1F249800AD
:101420000300000C4147432043572F5353423A20B7
:10143000FFF81F2498000400000941474320414D54
:101440003A2020FFF8FF1F2498000500000B532DC1
:101450004D74722063616C3A20FFF8FF1F249800DE
:101460000100000C464D2F494620746573743A20E4
:1014700002054F666620204F6E2020201F24980012
:10148000020000094F70656E2054783A2002084F20
:10149000666620202020204F6E202020202020FF64
:1014A0001F2498000300000D5443584F20547765C3
:1014B000616B3A2020FFF8FF1F2498000400000E03
:1014C0004D6963204761696E2063616C3A20FFF8C3
:1014D0001F24980005000008547820414C433A200E
:1014E00002094F66662020202020204F6E202020F9
:1014F000202020201F2498000100000E5478204452
:1015000072762043572F464D3A20FFF81F2498004B
:101510000200000E54782044727620414D2F534231
:101520003A20FFF81F2498000300000D5478205043
:10153000726F632043616C3A20FFF8FF1F2498000C
:101540000400000D54782053686628555342293A08
:1015500020FFF8FF1F2498000500000D5478205349
:101560006866284C5342293A20FFF8FF1F24980050
:10157000010000054D7367313A010CFF1F249800EC
:10158000020000054D7367323A010CFF1F249800DA
:10159000030000054D7367333A010CFF1F249800C8
:1015A000040000054D7367343A010CFF1F249800B6
:1015B000050000054D7367353A010CFF1F249800A4
:1015C000010000054D7367363A010CFF1F24980097
:1015D000020000054D7367373A010CFF1F24980085
:1015E000030000054D7367383A010CFF1F24980073
:1015F000040000054D7367393A010CFF1F24980061
:10160000050000054D7331303A010CFF1F2498008E
:101610000100000E436C722074756E6572206D655A
:101620006D3A0203204E6F5965731F249800020023
:1016300000084320287046293A2001F81F2498000A
:101640000300000E4320736964653A2020202020A7
:1016500020200203416E745478201F249800040057
:1016600000084C20286E48293A2001F81F249800D1
:101670000500000E466F72636520726574756E65B5
:101680003A2002034E6F205965731F249800010011
:101690000010507263312052657620422E30322E77
:1016A0003035010120FF1F2498000200000950720C
:1016B00063322052657620FFF8FF1F249800030054
:1016C000000A202020202020202020200207202087
:1016D0002020202020202020202020201F249800AF
:1016E0000400000A202020202020202020200207A3
:1016F00020202020202020202020202020201F24E7
:1017000098000500000E52652D70726F6772616D52
:101710002075503A0203204E6F5965731F248A00CA
:1017200007000004464470780000240033003E00A7
:101730004C0054005C008D00A900BC00CB000000F0
:10174000240033003E004C005400DB00140125014E
:1017500036014B010000240033003E004C005400D1
:1017600060016B01770186019701000024003300BE
:101770003E004C005400A901B301BD01C701D101D5
:101780000000240033003E004C005400DB01E50162
:10179000EF01F9010A020000240033003E004C0072
:1017A00054001B02270233023F024B0200002400B8
:1017B00033003E004C0054005C027C028F02B502F4
:1017C000C1020000240033003E004C005400CD0252
:1017D000FC020E03280339030000240033003E00FE
:1017E0004C005400490363036E0379039303000024
:1017F000240033003E004C005400A903BC03CA037C
:10180000FC032E040000240033003E004C00540072
:1018100060047104AC04E7042205000024003300D6
:101820003E004C00540033053F054B05560560054E
:101830000000240033003E004C0054006B057B0583
:101840008D059905A5050000240033003E004C00DD
:101850005400B705C305CF05DB05E70500002400EC
:1018600033003E004C005400F305FB0503060B0655
:1018700013060000240033003E004C0054001B06F9
:1018800023062B0633063B060000240033003E00EF
:101890004C005400430652065B066A0673060000BD
:1018A000240033003E004C005400820690069A0645
:1018B000AB06BC06FF010707FA050303FA040101A2
:1018C00020000704FB040101FB0301011E040707BC
:1018D0004E000707FB0601012F0001011F03010154
:1018E0001D001F1D1E000101FB0501013100030346
:1018F000310203031700FFFF1900FFFF3107010149
:101900004C0003021F0007040B00FFFF0700FFFF4E
:101910000900FFFF0D00FFFF0F00FFFF0100FFFFA9
:101920000300FFFF0500FFFF0000000000000000B3
:101930001700FFFF1800FFFF1900FFFF1A00FFFF4D
:10194000500701011E0103031F04030228001F109A
:101950001B00FFFF1C00FFFF32001F1630060101B5
:10196000270007044D000101280701012200070498
:1019700023007F5424007F5425000F08260007040D
:101980000E0001010F000F0010000F0811000F08DA
:1019900012000F0813000F0114000F0D15000F0D9A
:1019A00016000F0D000000002B00FFFF2C00FFFFB2
:1019B0002D00FFFF2E00FFFF5400FFFF3104010147
:1019C000310501014A00FFFF4B00FFFF3106010115
:1019D0003300FFFF3D00FFFF4700FFFF4900FFFF0F
:1019E0004800FFFF7600000077000000780000004C
:1019F000790000007A0000007B0000007C000000FD
:101A00007D0000007E0000007F0000002900010131
:101A10001B00FFFF290101011D00FFFF2902010139
:101A2000000000004F00FFFF000000000000000069
:101A30002A00010132003400360090009200DE00DE
:101A4000E000A401A601A801AA01AC01AE01B00109
:101A5000B201B401B601B801BA01BC01BE01C001B6
:101A6000001B77403E000102FFFF001E84803C0007
:101A70000102FFFF003567E03E00FFFFFFFF00357A
:101A8000C9883EFF010203040036EE803CFF0102DC
:101A90000304003875203EFF01FFFFFF0039FBC043
:101AA0003EFFFF02FFFF003D09003C000102FFFF77
:101AB000005156443D000102FFFF005194C43D0017
:101AC0000102FFFF0051E2E43D000102FFFF00516F
:101AD000F66C3D000102FFFF0052736C3D000102F5
:101AE000FFFF006ACFC03E00FFFFFFFF006B3168C1
:101AF0003EFF01020304006CB8083CFFFF02030430
:101B0000006D7B583EFFFF02FFFF006F63A03C00AB
:101B10000102FFFF009A1D203E000102FFFF009A14
:101B2000E0703C000102FFFF00D59F803E00FFFFF8
:101B3000FFFF00D601283EFF0102FFFF00D7E9703A
:101B40003CFF0102FFFF00D84B183EFF01FFFFFFE3
:101B500000D90E683EFFFF02FFFF00DAF6B03C003E
:101B60000102FFFF0113B2203E000102FFFF011539
:101B700038C03C000102FFFF01406F403E00FFFF04
:101B8000FFFF0140D0E83EFF0102030401437C80D7
:101B90003CFF010203040143DE283EFF01FFFFFF7B
:101BA0000144A1783EFFFF02FFFF01474D103C00BA
:101BB0000102FFFF017BCA903E000102FFFF017D91
:101BC00051303C000102FFFF01AB3F003E0001022B
:101BD000FFFF01B2E0203CFFFFFF030401C52FA07F
:101BE0003C000102FFFF1895189518951895189557
:101BF000189518951895189518951895189518957D
:101C0000189518951895189518951895189518956C
:101C100018951B991895FFB60F931F932F933F9319
:101C20004F935F936F937F93BF93AF9306B10093EE
:101C300011012898AA27B2E0129711F01B9BFCCF44
:101C4000289AAA27B2E0129711F01B99FCCF06B18F
:101C5000009312012898AA27B2E0129711F01B9B5B
:101C6000FCCF02E000931B0010E100915301012B17
:101C70000BB90E942E3529980E942E350E942E35D0
:101C800006B1299A06FD09C00091830200680093FD
:101C90008302002700936C00E4C0109111011F77AC
:101CA000125000911201000F111FB801000F111FF7
:101CB00040912D05442331F0000F111F4A9511F07A
:101CC000060F171F3327222717FD3FEF17FD2FEFB2
:101CD000000F111F221F000F111F221F000F111FC5
:101CE000221FA801B901000F111F221F400F511F11
:101CF000621F731F09E4400F00EC501F07E3601FD1
:101D00000FE0701F0FEF07B908B910E100915A01F9
:101D1000012B08B910E400915301012B0BB90E946B
:101D20002E3529980E942E350E942E35299A01E0E1
:101D300008B90E942E350E942E35289A0E942E3511
:101D40000E942E35289878B90E942E350E942E3593
:101D5000289A0E942E350E942E35289868B90E9434
:101D60002E350E942E35289A0E942E350E942E353F
:101D7000289858B90E942E350E942E35289A0E9424
:101D80002E350E942E35289848B90E942E350E9483
:101D90002E35289A0E942E350E942E3528982F9A8B
:101DA00000002F98442700915A0130914E0137FFCF
:101DB00013C04FEF3F7730934E0127E032170CF4FA
:101DC000232F20937C0000915A01087F132F175076
:101DD0001770012B00935A0108B910E400915301C8
:101DE000012B0BB90E942E3529980E942E350E9496
:101DF0002E35299A40FF0DC00E942E350E942E35A7
:101E00000E942E350E942E350E942E350EED009335
:101E10007A001091C7042091C8041695279516954D
:101E2000279530919802231729F0209398020027D4
:101E300000939A0200919A0200FD2091990200916C
:101E40009702021749F0209397020FEF00933E0488
:101E500012E008E50E948134002707B90FEF08B9A6
:101E6000289AAF91BF917F916F915F914F913F9170
:101E70002F911F910F91FFBE1895FFB60F931F93DF
:101E80002F930091D4020023B1F00091F2010230AF
:101E900091F000270093FB030093FC0300930204DE
:101EA0000093FF03009303040093000400930404D1
:101EB0000093010410C000918302002361F400919B
:101EC000FC03002341F410E20E940F3811E005FDED
:101ED0001FEF1093FC032F911F910F91FFBE1895D8
:101EE000FFB60F931F932F930091D4020023B1F0FC
:101EF0000091F201023091F000270093FB03009360
:101F0000FC03009302040093FF0300930304009377
:101F10000004009304040093010410C000918302A4
:101F2000002361F40091FB03002341F410E20E94BE
:101F30000F3811E004FD1FEF1093FB032F911F9149
:101F40000F91FFBE1895FFB60F921F920F931F932C
:101F50002F933F93AF93BF93CF93DF93EF93FF9371
:101F6000009183020023D1F10336C1F10130B1F1B8
:101F7000023019F00330F1F408C303950093830293
:101F800000915A01086010E40E940F3801EC0E9491
:101F90005F3800915A0110E40E940F38002707B9FA
:101FA0000FEF08B902E000931B0008E000936C00FB
:101FB000289AEBC200915A01086010E40E940F3881
:101FC0000E945F3802E000931B000EED00937A0040
:101FD000002700934E0100938302D7C2B0914004C2
:101FE000A0914104109729F01197B0934004A09359
:101FF0004104A091C802B091C702109729F011972F
:10200000A093C802B093C7020091FF0407FF0E948B
:10201000873500917E02002361F00A9541F400911A
:102020007D02002331F022240E94873502C00093F4
:102030007E020091480407FF17C010914904112344
:1020400099F406FD03C00027112707C010914A0428
:102050001A9532F410E2012714E62CE0209349048B
:1020600010934A040093480400914304002319F09C
:102070000A950093430400912F0400230AF06CC0DA
:10208000A0912604B09125041197A0932604B09343
:10209000250409F061C000912D04009325040091EE
:1020A0002E040093260400910605002309F014C0B5
:1020B000009102051091050503951395011711F480
:1020C00000910405009302050E9470390E946B493B
:1020D0000FEF0093490240C010E00E94E838302F13
:1020E00031702D911D910C91AF93BF9310902704E7
:1020F00000902804000E111E00E0201F301F3170D8
:102100003F932F931F920F9211E00E94E838302FD7
:1021100031702D911D910C910F900016002D0F9094
:102120000106102D0F900206202D0F900306302D72
:1021300049F044F03091290420912A0410912B0495
:1021400000912C04BF91AF910C931E932E930E918E
:102150000E7F3170302B3C93B0915108A091520802
:102160001097B1F01197B0935108A093520881F4E1
:102170000FEF0093490200930D040093F5030093C1
:1021800079030093B0020093890204E1009369018E
:10219000B091E806A091E906109749F11197B09324
:1021A000E806A093E90619F5F4E0E1EEAA27BB27BB
:1021B000D1E0C9EF22270E943135102F008101178D
:1021C00019F00E9438352FEF11963196219799F723
:1021D000222369F00027009345040CE00093440497
:1021E000A4EFB1E0B0934604A093470412C0B091AD
:1021F0004604A0914704109761F01197B0934604EC
:10220000A093470431F40FEF009345040CE00093D2
:102210004404B091EA06A091EB06109761F0119783
:10222000B093EA06A093EB0631F40FEF0093D402CB
:1022300001E00093BB032091200410912104009140
:102240002204322F312B302B79F0015010402040E6
:10225000209320041093210400932204012B022BCD
:1022600019F401E000931E0400917B02023321F077
:10227000039500937B0209C000917D02002329F49D
:1022800001E000937D020E9487353FEF00917602C6
:10229000002359F00A9500937602002399F410E286
:1022A0000E940F38009358010DC010E20E940F38B1
:1022B00002FF05C003FF03C00093580103C002E3FF
:1022C000009376020091E706002319F00A95009327
:1022D000E7060091540110915501011709F05CC007
:1022E000009156010F7B109157011F7B011731F0B0
:1022F0006624009156010074102BEAC000914C0234
:10230000002319F00A9500934C0200914F0100231D
:1023100009F078C011270E940F381091D00210FDEB
:102320000F7710FD10951093D00210917B0211339E
:1023300019F00F3F09F466C000241091F201123029
:1023400009F4009410911E0417FF116810931E04E5
:102350001091540120E81090BC0101281090BB019D
:10236000012800FC006810FC006407FF1227269576
:1023700006FF1227269505FF1227269504FF122730
:10238000269503FF1227269502FF1227269501FFA7
:102390001227269500FF122700915401012706FFFE
:1023A00002C016FD3E7F3093340407FF0AC000913F
:1023B00056010C70C9F421E017FF2FEF2093ED01B7
:1023C00013C004FF11C030913B0400913D04043060
:1023D0002CF414FD316014FF3E7F04C014FD3068FE
:1023E00014FF3F7730933B04109354011093550131
:1023F00010955090590110935901012F10E30E943C
:102400000F38A4C010E10E940F38202F00741091E3
:1024100056011F7B012B0093560100914F010023B1
:1024200009F095C0022F0F7B3091340410FF032375
:102430003FEF309334041091D10210FD0B7F10FD5B
:1024400010951093D1021091D20210FD077F10FD5C
:1024500010951093D2021091BD0110FD0E7F10FD5A
:1024600010951093BD0110917B02113319F00F3BB1
:1024700009F470C000241091F201123009F40094A4
:1024800010911E0417FF116810931E04109156013D
:1024900020E866241090BC01012809F00C6100902E
:1024A000BB0100FC016007FF60942695269505FF9F
:1024B0001227269504FF1227269503FF122726953B
:1024C00002FF1227269501FF1227269500FF1227EB
:1024D0001093560110935701109550905C01109382
:1024E0005C01012F10E60E940F38662019F02FEFD3
:1024F0002093EB020091FF04087041F500915C010C
:102500000525087029F001E053FE0FEF0093E90163
:1025100000915C010525047029F001E052FE0FEFE7
:102520000093EB0100915C010525027079F051FEEA
:1025300003C00E94083307C000270093EA060093F7
:10254000EB060093D4020FEF0093BB0306E90A9554
:1025500000934F01009174020023B9F400915801D7
:10256000007410917502102710E069F010E20E94CB
:102570000F38202F00740093750211E0207C11F0B9
:10258000203C09F41FEF1093740200EE06BDFF918A
:10259000EF91DF91CF91BF91AF913F912F911F911B
:1025A0000F911F900F90FFBE1895FFB6AF93BF938A
:1025B0000F931F932F930091F406002319F00091BD
:1025C000C60031C0B6E0A6EF1091F5060027A10FB6
:1025D000B01F0091C600003234F10C931395209186
:1025E0002E052223A1F0163440F02091CD0220FDCB
:1025F0000EC021682093CD020AC01A3040F4209109
:10260000CD0220FD04C02E7721602093CD0210352D
:1026100011F01093F5060B3331F40FEF0093F4062D
:1026200000270093F5062F911F910F91BF91AF9155
:10263000FFBE1895FFB6AF93BF930F931F93009102
:102640004607002331F40091C1000F7D0093C100C3
:102650000EC0B7E0A8E410914707101B0A9500933D
:1026600046070027A10FB01F0C910093C6001F91D1
:102670000F91BF91AF91FFBE1895FFB60F921F92B9
:102680000F931F932F933F93AF93BF9300917800C5
:102690001091790020914E012C3021F43FEF3093BE
:1026A000CF0257C02730D1F43091CB02332309F445
:1026B00050C0313019F42227209325010E94FC4C90
:1026C00019F4383C31F002C0323119F033953093AF
:1026D000CB02B1E0A6E32091250133C02830C9F533
:1026E0003091CB023230A8F10E94FC4C19F4383CF6
:1026F00051F002C0323139F0002433953093CB02CF
:10270000383C09F4009430912101209122010217F4
:10271000130772F0112341F40E3634F4002041F017
:1027200036EC3093CB0204C01093210100932201B8
:10273000B1E0A6E230912501232F33953770309315
:102740002501220F3327A20FB31F1D930C93209155
:102750004E012F93220F3327A3ECB4E0A20FB31F37
:1027600011962695273084F411971D900C903327ED
:1027700023E0200D311D0217130734F4900122507D
:1027800030400217130714F40C931E932F912395D6
:102790002F3021F422270FEF0093D70220934E0110
:1027A00000918302002321F0206820934E011EC077
:1027B00007E020170CF4022F00937C0007305CF038
:1027C00000915A01087F27502770022B00935A016D
:1027D00010E40E940F3800914E01073024F00E944F
:1027E0002E350E942E350EED00937A00BF91AF91E9
:1027F0003F912F911F910F911F900F90FFBE189541
:10280000FFB6209083022220A9F420907D0222208E
:1028100089F00F921F920F931F932F93EF93FF93C3
:1028200022240E948735FF91EF912F911F910F91E4
:102830001F900F90FFBE189500E10EBF0FEF0DBF68
:1028400000E002B9002701B90EE405B90093520176
:1028500003EF04B90FEF08B9009507B90FE00BB902
:102860000093530102EF0AB9A0E0B1E0EBEBF8E00E
:10287000EA1BFB0B00270D933197E9F70FEB009351
:1028800056010FEF0093590100935C01B5E7A0E3F7
:10289000B0934004A09341040093190400934701AE
:1028A00001E00093A90200934A020093F7030FE7A7
:1028B0000093EC060AEA0093C3040093C40400ECFE
:1028C00000935A0100E800931E0408E000935B01A6
:1028D0000AE00093A4020093A702E8EDF5E0AAE65F
:1028E000B1E005E10E94C238EEEEF5E0AFE7B1E0FD
:1028F00007E20E94C238E2E4F6E0AEEBB1E00DE0A0
:102900000E94C238E0E9F6E0A6EAB1E00DE00E94DC
:10291000C238EEE9F6E0A8EDB2E00DE00E94C23860
:10292000E6E3F5E0ACEEB2E00EE00E94C238E8E289
:10293000F5E0AEE4B3E00EE00E94C238E6ECF6E06B
:10294000ACE5B3E007E10E94C238E4E4F5E0ABE7B0
:10295000B3E00CE00E94C238EAEBF6E0A9E9B3E08C
:102960000BE00E94C238EEEDF6E0ACEBB3E00FE016
:102970000E94C238EEEEF6E0ABECB3E007E10E9455
:10298000C238E2E4F7E0A4EEB3E000E10E94C2380E
:10299000EEEBF7E0A8E3B8E00CE00E94C238E6EA0C
:1029A000F7E0A4E5B8E007E10E94C23800915B01BE
:1029B000016010E50E940F3800915B010E7F10E569
:1029C0000E940F3804E11DE128E20E948B3804E1E7
:1029D0001DE120E20E948B380AE41EE128E20E94F9
:1029E0008B380AE41EE120E20E948B3800271FE1A9
:1029F00028E20E948B3800271FE120E20E948B38DA
:102A000000E410E228E20E948B3800E410E220E2A9
:102A10000E948B3801E020E10E94443801E028E365
:102A20000E94443801E020E30E94443801E028E19C
:102A30000E9444380E944132002707B9009508B926
:102A4000F4E0E1EED1E0C9EFBB27AA270E943135BF
:102A5000019311962197D1F70E94703900270093B6
:102A60000B0500912F050093C4023327222711275D
:102A7000009102055FEF48E00E9445320091DA01C3
:102A80000093A503009315040091DB010093A603B6
:102A90000093160410E00E94E8380E7000933C0486
:102AA000102F0091FF0403FD1091E2041E7010939B
:102AB0003D0411270091EE0407FD18E000FD1460AD
:102AC000109357010E94F938037011272091FF04D9
:102AD00023FD1068002339F01260013021F01160ED
:102AE000023009F013601093550101E300933F0495
:102AF00005E00093240408E00093E0060CE4009352
:102B0000E1060BE40093E20600E40093E3060027ED
:102B10000093E4060093E506009109050078009310
:102B20001D0491F404E1009369010FEF0093490241
:102B300000930D040093F503009379030093B00212
:102B4000009389020093340400912B0515E0019F46
:102B5000800123E033270E94BF490093390410937A
:102B60003804222711270027309112053C7030933A
:102B70001F0469F026E01DED00ED343041F02DE03A
:102B80001BEB00EA303119F02BE117E700E420934A
:102B90002004109321040093220403E000937C009E
:102BA0000EED00937A0000270093C50010910805F0
:102BB00007E6112351F003E3113039F009E1123037
:102BC00021F000E1133009F008E00093C40008EBA5
:102BD0000093C10006E00093C20000912E0500237F
:102BE00019F001E80093CD0200EE06BD05E005BD39
:102BF00001E000936E000FE30093690007E00DBB56
:102C000002E000936800B3E0A8EE1B9902C01197A0
:102C1000E1F700915A01086010E40E940F38002784
:102C20000E945F380E945F380E945F380E945F38C0
:102C30000E945F380E945F380E945F380E945F38B0
:102C40000E945F380E945F380AEA0E945F38009154
:102C50005A0110E40E940F380FEF08B9002707B996
:102C60000E947738053529F00CE10093800200932B
:102C70008102789400918102002309F0FACF00913B
:102C8000D7020023B1F300918302002359F00336E9
:102C900031F0013071F7039500938302EACF01E030
:102CA000009383020091C902002381F400910B0577
:102CB0000023A9F0F8940FEF0093C902B3E1A8E84C
:102CC000B093C702A093C802789409C0F894B09159
:102CD000C702A091C802109711F40C94007E0091D5
:102CE0001D040023E9F00091530810911904012BF1
:102CF000B9F4B7E0A8E9F8E0E4E41CE00D91019331
:102D00001A95E1F7B9E0A4ECF894B0935108A093B8
:102D10005208789408E1009350080FEF009353088D
:102D2000F894B0914004A0914104BA2B59F4209139
:102D30005A012F7B10E40091110500740127022B2A
:102D400000935A01789400914902002331F40E94C3
:102D50000E3A00914B02009349020091BA030023FE
:102D6000D9F44091BB0340FF17C00CE41FE623E6F3
:102D70003BE647FF03C000E2102F98010093C70312
:102D80001093C8032093C9033093CA030FE0009344
:102D9000BA0300270093BB0300912F040023FAF429
:102DA0000091220017E1019F02E7000D1091E0045D
:102DB0001017A8F0F8940027009325040093260428
:102DC000039500932F042091D60204E516EA0E9491
:102DD00081342091D50204E515EA0E9481340091E6
:102DE0001E0400FFB5C00E7F00931E0407FF66C0DF
:102DF00001E00093F70303E00093F6032091D6026D
:102E000004E516EA0E9481342091D50204E515EA12
:102E10000E9481340091C40200932F0504E11DE15A
:102E200028E20E948B3804E11DE120E20E948B38E9
:102E300001E020E10E94443801E028E30E94443888
:102E400001E020E30E94443801E028E10E94443878
:102E50000E9441320091630110EC0E942B380091D6
:102E60005D0110E70E942B380091640110ED0E9473
:102E70002B382091320510E50EE90E94813422277B
:102E800011270027309112053C7030931F0469F020
:102E900026E01DED00ED343041F02DE01BEB00EAA3
:102EA000303119F02BE117E700E4F8942093200467
:102EB000109321040093220478944AC000270093C1
:102EC000F70303E00093F603222704E516EA0E94C5
:102ED0008134222704E515EA0E94813400912F05F0
:102EE0000093C402002700932F0507E128E20E9407
:102EF0008B3807E11DE120E20E948B3804E020E1DD
:102F00000E94443804E028E30E94443804E020E3AF
:102F10000E94443804E028E10E9444380E94413273
:102F2000009163010C7F10EC0E942B3800915D0131
:102F30002B7F10E70E942B380091640100640F7D05
:102F400010ED0E942B382FEF10E50EE90E9481341E
:102F50000091F503002309F46CC00091F4030023F1
:102F600009F067C000270093F50300912F040023A8
:102F700031F043E533E421E41EE400E24DC000916A
:102F80003004002331F040E23DE425E41DE400E29A
:102F900043C00091E104222723950550EAF70A5F18
:102FA00010E3010F1DE2213021F441E336E320E379
:102FB00033C0223021F440E238E320E32DC0233037
:102FC00021F440E236E320E327C0243021F440E23C
:102FD00034E320E321C0253021F440E233E320E351
:102FE0001BC0263021F440E232E320E315C0273035
:102FF00021F440E231E327E30FC0283021F440E21E
:1030000031E325E309C0293021F440E231E322E332
:1030100003C040E231E320E34093EF033093F00339
:103020002093F1031093F2030093F30300E1009364
:10303000F4033091AC020091CF02002309F477C071
:10304000F89400270093CF021091DB040091DC0478
:10305000789416950795169507950C3D08F067C06E
:10306000033C30E0A0F431E0053A88F432E0073860
:1030700070F433E0093658F434E00B3440F435E0B2
:103080000D3228F436E00F3010F437E050C00091D4
:10309000AC023093AC020630A1F4363091F00091CE
:1030A0003704002371F4002700933504E6EAF7E0C3
:1030B000A4E5B8E007E10E94C23807E100933704B5
:1030C00036C0343041F000912F04002321F0002756
:1030D00000932F040BC0353051F1009130040023D0
:1030E00031F10027009330040E943E4A10E00E9414
:1030F000E838309129043E933E7030933C040091AF
:10310000FF0403FF30933D0420912A0410912B0407
:1031100000912C0411962D931D930C930FEF0093A7
:10312000F5030093790300930D0400934902009185
:10313000EB02002309F400C100270093EB02009189
:10314000F201023009F4E3C03091AC0234300CF4E7
:10315000CCC0343009F41DC0353009F4A4C0363079
:1031600009F0EAC000913504002341F400913604CF
:103170000E94694A0FEF00933504DEC000913D04C0
:1031800004300CF0D9C000913604039500931C0460
:10319000D3C0F89400912F04009500932F0492F06F
:1031A00001E000932F042091D60204E516EA0E9464
:1031B000813478942091D50204E515EA0E94813487
:1031C0007894BAC00E3F71F010E00E94E838009386
:1031D00029040D9100932A040D9100932B040D9165
:1031E00000932C04789400910605002309F00EC08A
:1031F000F894009104050093020578940E947039B8
:103200000E946B490FEF0093490223C0009106050D
:1032100022271AE00130C9F014E60230B1F023E0B1
:1032200018EE033091F027E210E1043071F02AE348
:1032300018E9053051F02EE410E2063031F021E6B5
:1032400018EA073011F023EC10E5209327041093BF
:10325000280400910705222712E3002361F01DE7EF
:10326000013049F01AEF023031F021E014EF033061
:1032700011F029E014ECF89420932504109326040F
:1032800020932D0410932E047894222704E516EA47
:103290000E948134222704E515EA0E9481340FEF51
:1032A0000093F50349C010E00E94E8380093290418
:1032B0000D9100932A040D9100932B040D9100931E
:1032C0002C0400913004002331F00E946B490FEF71
:1032D0000093490231C00FEF009330040093F503CF
:1032E0000E9470390E94A33927C000916F02009597
:1032F00000936F020AE210E211F000E21AE200937A
:103300006703109370030FEF0093790315C00091CA
:10331000F1010E3011F00F3079F41091F3011630F5
:103320005CF000911A0403950C3009F40027009317
:103330001A040FEF00931704F8940091CB020023B6
:10334000B9F40093920300939303009391030093C5
:1033500021010093220100930301009304010093D3
:10336000050100930601009301010093020106C0CC
:103370000E94E04B0E94FE4B0E94364CF894109144
:10338000D5040091D6047894000F111F0654104004
:1033900000930C0110930B010091FF0406700430A0
:1033A00029F0063019F00027112714C0F894109165
:1033B000DD040091DE047894000F111F000F111F2F
:1033C000000F111F000F111F000F111F33272AE0DC
:1033D0000E94BF490093080110930701F8941091CF
:1033E000D7040091D80478941695079500930A01A4
:1033F00010930901F8941091D9040091DA0478949B
:10340000222733274091FF04542F4077403209F0A0
:1034100037C05670563039F41695079516950795AE
:103420001695079525C0F8941091030100910401A9
:103430007894000F111F000F111F3327209189026C
:103440004091FF04467029F0423019F03AE0239F82
:103450009001432F422B09F423950E94BF49980104
:1034600036952795020F131F11F4073608F007E66B
:10347000009394033327222714E6019F800104C0A0
:10348000202F312F002711270093100110930F01D7
:1034900020930E0130930D01222700911E0407FF97
:1034A0000BC0009156010093840206FD2068009134
:1034B0004204002309F0206810913B0400913D0470
:1034C00004303CF00A3009F42062206417FD05C086
:1034D0000AC010FD206210FF06C0F894009154014C
:1034E00004FD0AC005C0F8940091540104FF04C013
:1034F00010E1012700935501789400915C0105FFCC
:10350000206100910005007306950695202B10910F
:103510000105177029F01A95212B2093CE0215C0B2
:1035200000914204002329F5F89400915A010860A3
:1035300010E40E940F3806ED0E945F3800E8009307
:1035400042040E945F38789414C000914204002322
:1035500081F0F89400915A01086010E40E940F383D
:1035600006ED0E945F380027009342040E945F38F6
:1035700078940091FF04067009F4ECC10091C00238
:1035800020912C0510914701112311F4021731F0FD
:103590002093C002112708E50E948134789400919D
:1035A0003D040A30C9F00091B2022091F904109153
:1035B0004701112351F410913E04112321F00027FB
:1035C00000933E0402C0021739F02093B20212E0C9
:1035D00008E50E94813478940091FF040078B9F0E6
:1035E000F8941091C7042091C804789416952795F3
:1035F0001695279500914701002391F43091980288
:10360000231729F020939802002700939A02009133
:103610009A0200FD20919902009197020217A1F0F1
:103620002093970200913D040A3029F40FEF009394
:103630003E0412E005C00E94F93813E005FD11E0D8
:1036400008E50E94813478942091A1020091FF0442
:10365000007851F0F8943091CF042091D004789400
:10366000369527953695279536952795369527953E
:103670003AE7230F0091FF04007849F03091A0024F
:10368000231729F02093A00200270093A2020091A3
:10369000A20200FD2091A10200913B0407FD09C098
:1036A000209128052A3710F42AE703C02A3B08F0A6
:1036B00029EB00914701002321F400919F0202179A
:1036C00039F020939F0216E50EE90E948134789428
:1036D00000270093460120918C020091FF0400789E
:1036E00051F0F8943091CD042091CE047894369521
:1036F0002795369527950091120506FD08C021955E
:103700002A3F20F4263310F0209332052195269588
:103710001091FF04107849F010918B02121729F0D4
:1037200020938B02112710938D0210918D0210FDB2
:1037300020918C0200918902021729F4009147011F
:10374000002309F432C0209389020091E90200238A
:1037500061F546E00091FF04067019F0023009F0AF
:1037600047E033272227009189021AE0019F800158
:1037700055270E944532A5EEB2E00091D8010D9385
:103780000091D9010D930091DA010D930091DB01B5
:103790001091FF04167019F0123009F000E20C933A
:1037A00001E10093E902009346010091840206FDC5
:1037B00007C000914204002319F40093CB02CAC051
:1037C00000913D04003019F0023009F01EC0F89459
:1037D00000915A01086010E40E940F3805EC0E9425
:1037E0005F3800915A0110E40E940F380FEF08B9BA
:1037F000002707B90E9477387894002331F4F894B1
:1038000000270093CB027894A5C0F8940091CB02D6
:10381000002351F478940AE00E94C74BF89401E029
:103820000093CB02789496C078942091120526FFDD
:1038300057C00E94FC4C51F4083C09F08BC0109119
:103840002101009122010E941C4C07C0023109F0A5
:1038500081C0109103010091040133272AE04091B7
:10386000FF04467019F0423009F024E60E94BF4977
:103870001091890216C0309191033A5190F041E1C4
:10388000349F80012AE033270E94BF4910918902AA
:103890003FE7301B37FD332700918E02311708F4C4
:1038A000132F21E0101B10F4119521953091240461
:1038B000131728F400914601002309F44BC010911E
:1038C0003205121B1A3F48F4163318F010933205D4
:1038D00007C019EF1093320503C016E310933205A9
:1038E00013E300913D04003029F0023019F00A3052
:1038F00009F01DE30E94CE38202F2A3710F42AE762
:1039000003C02A3B08F029EB44270091C6020217A6
:1039100041F02093C60212E50EE90E9481347894AA
:103920004FEF0091C50220913205021741F020931C
:10393000C50210E50EE90E94813478944FEF4423CC
:1039400049F0F89400270093210100932201039588
:103950000093CB02789400913C040A3011F420ECDF
:1039600044C00091FF040078C1F0F8941091C9049C
:103970000091CA0478949801369527953695279535
:1039800030919C02321729F020939C023327309308
:103990009E0230919E0230FF07C0112700919D02C8
:1039A000000F111F000F111F1095009513702BEEC3
:1039B00035E0020F131F20910C0540915F0143FD7C
:1039C00020910D053327220F331F220F331F220FA3
:1039D000331F220F331F200F311F36952795369541
:1039E000279536952795369527954427009100050C
:1039F000087089F402E4013421F000913D040430A0
:103A000054F00091560106FD04C0009142040023C9
:103A100011F020EC406200919B02109147011123AC
:103A200011F4021739F020939B0214E10EE90E9471
:103A30008134789420915B012971009131050078DF
:103A4000202B00911E040095007806950695202BEA
:103A50000091C302202B02E4013451F02F7D00912C
:103A60003D0404302CF000911E0407FF01C0242BFC
:103A700010914701112321F410915B01211741F0AE
:103A8000F89420935B01022F10E50E940F38789480
:103A9000209135050091BE0210914701112311F4C8
:103AA000021739F02093BE0210E50CE90E94813420
:103AB0007894209134050091BF02109147011123A1
:103AC00011F4021739F02093BF0212E50CE90E94AD
:103AD000813478940091FF04007899F0F894309143
:103AE000CB042091CC04789436952795369527956C
:103AF00030919402231729F0209394020027009319
:103B000096020091960200FD209195022695269539
:103B1000269500914701002321F40091930202179A
:103B200061F02093930200E515EA0E9481347894B5
:103B300000E516EA0E94813478940091FF04007831
:103B400099F0F8943091C5042091C6047894369584
:103B500027953695279530919002231729F02093C9
:103B600090020027009392020091920200FD2091A2
:103B7000910226952695269500914701002321F470
:103B800000918F02021759F020938F0202E515EA87
:103B90000E948134789402E516EA0E948134789478
:103BA00011270091590102FF13C003FF22C0209189
:103BB000D602222321F42FE12093D6021FEF209179
:103BC000D502222331F52FE12093D5021FEF21C02A
:103BD0002091D602222321F022272093D6021FEF24
:103BE0002091D5022223A9F022272093D5021FEF8E
:103BF00010C02091D602222321F42FE12093D60277
:103C00001FEF2091D502222321F022272093D502F5
:103C10001FEF00914701002311F4112369F0209157
:103C2000D60204E516EA0E94813478942091D502E8
:103C300004E515EA0E94813478942091FF042078ED
:103C400099F0F8943091C3042091C4047894369587
:103C500027953695279530918602231729F02093D2
:103C600086020027009388020091880200FD2091BF
:103C7000870200914701002321F400918502021779
:103C800031F02093850216E10EE90E948134789488
:103C90002091AC02222329F44091740240937A03CC
:103CA000DBC024300CF486C0243009F44BC025302E
:103CB00029F1263009F0D0C0009135040023D1F05D
:103CC0000091360410917402112331F032F40A95F8
:103CD000002342F409E006C0BFC0102F03950A304C
:103CE0000CF0002710913704112321F400933604BF
:103CF0000E94694A002700937402AEC0F8940091B4
:103D000030040023D9F000910205109174021123B0
:103D100039F03AF40F770A9500234AF404E507C016
:103D20009BC0102F0F77039505350CF000270093EB
:103D3000020578940E9470390E94A33900270093ED
:103D400074028AC000912F04002379F1F894009145
:103D5000070510917402112389F00091F2010230DD
:103D600009F423C0112322F40A954AF4002707C05E
:103D70000395043024F019F004E001C06DC00093F5
:103D80000705222712E3002361F01DE7013049F007
:103D90001AEF023031F021E014EF033011F029E086
:103DA00014EC20932D0410932E040027009374022A
:103DB000789452C00091EA02002309F04DC040916E
:103DC0006F0200917702442311F000917802409134
:103DD0007402442329F012F0039509C00A9507C024
:103DE0002091790227FF38C02F772093790212E3C0
:103DF000213021F014E6223009F01AEF002372F48A
:103E00000C3E0AF40CEE0195019F0094109411E011
:103E1000010E10E0111E1FEF019505C005310AF0DB
:103E200004E1019F112740916F02442359F400934C
:103E30007702109305041093060410920704009271
:103E400008040AC0009378021093090410930A042E
:103E500010920B0400920C040E94F938212F1C715F
:103E600016951695312F00913C04083009F4306204
:103E70002076203039F0203419F0203639F007C090
:103E8000386005C004301CF0386001C0306110910A
:103E90000005187011F0306401C03F7B1091FF04E1
:103EA000117009F0306800914701002321F410914E
:103EB0005F01311731F030935F01032F10E90E9449
:103EC0002B3820EA00913C040A3011F42F7D206544
:103ED00000917A030023B1F01091730240916F02B8
:103EE00040FF10917202010F12F403E003C004308E
:103EF0000CF00027442319F00093730212C00093C2
:103F000072020FC010E00E94E838007F0295102F67
:103F1000037000937202012F0695069503700093BB
:103F200073021FE000917202100F0E94CE383327F7
:103F300010917002101719F03FEF009370021AE011
:103F4000019FECE7F0E0E00DF11D3596AAE6B3E045
:103F500005910D9305910D9305910D9305910D9389
:103F60001596BF93AF933F9313E100917302100F27
:103F70000E94CE383F9110917102011719F03FEF66
:103F800000937102AF91BF911AE0019FE0E5F2E06A
:103F9000E00DF11D359605910D9305910D93059159
:103FA0000D9305910D9300917903032B51F000912E
:103FB0007803002331F40CE1009378030027009389
:103FC000790300917302000F000F10917202102B01
:103FD0001F9300917A03002399F0002700937A033E
:103FE00010E00E94E8380F701F911F931295012B6B
:103FF000F8940E930E94C73878940FEF00930D0445
:104000001F91212B00914701002321F410916001A1
:10401000211731F020936001022F10EA0E942B3803
:104020000091EA02002309F071C00091590106FFD6
:104030006DC000917402002321F0002700937402E8
:1040400008C000910D04002309F460C0002700930C
:104050000D04409170020AE2409FE6EDF0E0E00DB1
:10406000F11DAAEFB2E00AE20E94C238409171024B
:104070000AE2409FECEDF2E0E00DF11DA4E2B3E0B6
:104080000AE20E94C2380091770210910003100FDB
:104090001093000310910403100F10930403109168
:1040A0000E03100F10930E0310911203100F1093B4
:1040B000120310911C03100F10931C031091200386
:1040C000100F109320030091780210912A03100F13
:1040D00010932A0310912E03100F10932E031091AA
:1040E0003803100F1093380310913C03100F1093F6
:1040F0003C0310914603100F1093460310914A039E
:10410000100F10934A0300E70093EA020091B903ED
:104110000023E1F41091FF041077129500914701FC
:10412000002329F40091B002011709F40FC0109385
:10413000B0020AE0019FF5E0E0E5E00DF11DB3E01B
:10414000A7E80E94C23806E10093B9030091FF047A
:104150000077003009F420C0003109F42CC000328F
:1041600009F437C0003309F437C0003409F437C00C
:10417000003509F437C0003609F437C0F8941091BF
:10418000D7040091D80478942CE333270E94BF49C8
:10419000202F0093970340C0F8943091D5042091CC
:1041A000D604789436952795369527953695279594
:1041B0002093960331C0F8941091D9040091DA0449
:1041C00078942AE033270E94BF49202F009395035B
:1041D00023C02091940320C0209191031DC0209101
:1041E00092031AC02091930317C0F894109107010D
:1041F00000910801789416950795169507951695E0
:10420000079516950795169507952AE033270E947E
:10421000BF4900939803202F00914701002321F408
:104220000091AF02021731F02093AF0210E10EE9C6
:104230000E94813478940091FF04067009F407C14C
:1042400000913D04222704305CF008306CF0A1F0AE
:104250000A3041F40E94F9380072A9F0206813C0B6
:10426000206811C028690FC020610E94F9380072CF
:1042700009F02068286007C020620E94F9380072A7
:1042800009F0206828601091FF041670163009F4B8
:1042900024600091120507FD216000913D04083063
:1042A00009F421602F930E9405393E9131701196D7
:1042B0002D911D910C9170E06EE154E840E80E9450
:1042C000B5382F910CF422600091FF040077003282
:1042D00009F4206400914701002321F410915D014D
:1042E000121731F020935D01022F10E70E942B3846
:1042F0000E9405393E91317011962D911D910C91BE
:10430000882740915D0141FD1CC070E06BE55DE8D0
:1043100040E80E94B53814F4806113C070E067EB88
:104320005BE140E00E94B53814F480620AC071E09D
:1043300061E35DE240E80E94B53814F4806401C096
:10434000806870E066E255E240EA0E94B53814F4F5
:1043500021E049C070E06CE45BE440E40E94B538C1
:1043600014F422E040C070E063E55CEE40E60E9499
:10437000B53814F4222737C070E062E750E740EE0A
:104380000E94B53814F423E02EC070E067EB5BE1C7
:1043900040E00E94B53814F424E025C070E064EFDA
:1043A00054E240E00E94B53814F425E01CC071E0EE
:1043B00061E35DE240E00E94B53814F426E013C0EA
:1043C00071E06FE451EB40E80E94B53814F427E047
:1043D0000AC071E06BEA5FE340E00E94B53814F474
:1043E00028E001C029E02093C202822B00914701FE
:1043F000002321F410915E01811739F080935E0152
:10440000F894082F10E80E942B388695869586959B
:104410008E7109F4816080640091FF04067021F0C0
:10442000023011F080628F7B00911E0400950078AD
:10443000802B00914701002321F410916401811722
:1044400031F080936401082F10ED0E942B380E94F8
:104450000539222713960C91087009F020683FE770
:1044600044270091540105FF61C0822F0E911E91D7
:104470002E913E913170110F221F331F4427552773
:104480006EE1B4E0ABE40EE1061B000F000F112754
:10449000A00FB11F1D9117FD04C050FF962F5FEFB5
:1044A00011C013700D910217130761F40D911C9147
:1044B000712F782777FD06C04FEF0093ED061F7729
:1044C0001093EC066A95E9F650FF9EE100915601C3
:1044D00006FF27C000910A0502FF04C00B7F00936E
:1044E0000A0502C04423E9F42F933F938F939F93CF
:1044F0000E94B44A9F918F913F912F91B4E0ABE419
:104500000EE1091B000F000F1127A00FB11F30682B
:104510003D932D930091ED060D930091EC06082B31
:104520000C93282F3091EC064091ED0664E057EA99
:1045300046FD02C05A50604045FD02C054516040E3
:1045400044FD02C05752604043FD02C052556040D6
:1045500042FD02C05659604041FD02C05A546140BC
:1045600040FD02C05053624060931B0150931C01F8
:1045700000910A050D7F47FD026000930A0566E27F
:1045800058EE36FF02C05651604035FF02C052530C
:10459000604034FF02C05A58604033FF02C0565298
:1045A000624032FF02C0585D644031FF02C05E5677
:1045B0006A4030FF02C05A5A644160931D01509313
:1045C0001E01232B00914701002321F41091660165
:1045D000211731F020936601022F10EF0E942B3833
:1045E000242F00914701002321F410916501211728
:1045F00031F020936501022F10EE0E942B3880E1EC
:1046000000915901037049F0023029F0013039F46A
:1046100084608F7E04C0816001C0836080620E94DC
:10462000F9380C7F1127803139F01395843021F04F
:104630001395813309F01395012B0E93007109F046
:10464000806410910005187009F0806410E00E94E9
:10465000E838302F31702D911D910C9170E069E197
:1046600050EF40EA0E94B5380CF080680091470195
:10467000002321F410916301811741F080936301BD
:104680000E94C738082F10EC0E942B3820910F058C
:1046900000915F01007211F420910E050091470115
:1046A000002321F40091AE02021731F02093AE02F4
:1046B00012E10EE90E9481340E94F938007419F069
:1046C00080E89FE76AC088279FEF10E00E94E838E3
:1046D000302F31702D911D910C9170E06BE157E7F7
:1046E00040E40E94B53814F49B7F57C070E06DE23F
:1046F00056EC40EC0E94B5381CF484609B7F4DC0A2
:1047000070E06DE359E040E00E94B53814F4977F03
:1047100044C070E066E65FEF40E30E94B5381CF4E9
:104720008860977F3AC070E069E854E540E40E94F1
:10473000B53814F49F7E31C070E060EA57E340EA78
:104740000E94B5381CF480619F7E27C070E06FEA3C
:1047500059E740EE0E94B53814F49F7D1EC070E00A
:1047600064EF54E240E00E94B5381CF480629F7D03
:1047700014C071E061E35DE240E00E94B53814F4DA
:104780009F7B0BC071E06DE758E740E40E94B538AD
:104790001CF480649F7B01C09F7700914701002338
:1047A00041F400916101081721F400916201091799
:1047B00061F08093610190936201082F10EB0E94D9
:1047C0002B38092F10EB0E942B3822270091F80478
:1047D0001091B102011719F02FEF0093B10200916F
:1047E000FA041091B302011719F02FEF0093B302EE
:1047F0000091FB041091B402011719F02FEF009300
:10480000B4020091FC041091B502011719F02FEFCA
:104810000093B5020091FD041091B602011719F042
:104820002FEF0093B6020091FE041091B70201171A
:1048300019F02FEF0093B702009109050F71109145
:10484000AD02011719F02FEF0093AD020091A40201
:104850001091A302011719F02FEF0093A30200910A
:10486000A7021091A602011719F02FEF0093A602DC
:1048700000912F051091BB02011731F02FEF00932B
:10488000BB0203E00093F60300911C04002309F02F
:104890002FEF0091CE021091B902011719F02FEFFE
:1048A0000093B90200912D051091BA02011719F079
:1048B0002FEF0093BA0200914701202B29F40091B9
:1048C0001804002309F485C0F8942F9300915A012D
:1048D000086010E40E940F381091F8040091180449
:1048E000002369F00AED0E945F3810EAD7E0C8E9BA
:1048F00009910E945F381A95D9F7109318042F91E7
:10490000222309F45DC005ED0E945F380091F80490
:104910000E945F380091FA040E945F380091FB0406
:104920000E945F380091FC040E945F380091FD04F2
:104930000E945F380091FE0403950E945F38009149
:1049400009050F7111F014E0010F0E945F3800910A
:10495000A502002311F00091A4020E945F3800918B
:10496000A802002319F00091A70203950E945F3866
:104970000091BB020E945F3800911C04003839F49A
:1049800002E000931C040A950E945F3805C00E9453
:104990005F38002700931C040091CE020E945F380C
:1049A0000091CE02007E003E39F400918302002384
:1049B00019F403E60093830200912D050E945F38ED
:1049C0000091510810915208012B19F4002700930F
:1049D0004701F89400915A01086010E40E940F38D2
:1049E000009119040023D9F004EC0E945F38009173
:1049F0005A0110E40E940F380FEF08B9002707B9D9
:104A000010EAD7E0C8E90E94773809931A95D9F7D8
:104A1000109319040E947738009330056BC002ECA4
:104A20000E945F3800915A0110E40E940F380FEF86
:104A300008B9002707B90E94773800931F010E9428
:104A40007738009320010E947738009315010E9467
:104A50007738009316012091FF042F7710911501EC
:104A600017FD20682093FF041F771093150127FD81
:104A700014C00FEF0093880200938D020093A202EE
:104A8000009392020093960200939A0200939E0272
:104A90000093A5020093A8022DC03091BC02209182
:104AA0002001231789F02093BC0233273093A502FD
:104AB000222309F423E114E003E90E94BF49009393
:104AC0001A0100270093190120911F010091BD02D6
:104AD000021781F033273093A8022093BD022223CE
:104AE00009F420E21AE702E10E94BF49109317017E
:104AF0000093180110911501009116012091CD022B
:104B00002F7B16FD20642093CD021F7326FF16C055
:104B100020FF14C02E7F2093CD021F930F9300918E
:104B20005A01086010E40E940F380FED0E945F38B0
:104B30000091CD020E945F380F911F912091540186
:104B400026FD73C1169507951695079511E001335B
:104B500010F112E00134F8F013E00135E0F014E058
:104B60000136C8F015E00137B0F016E0013898F0D2
:104B700017E0013980F018E0013A68F019E0013BD4
:104B800050F01AE0013C38F01BE0013D20F01CE041
:104B9000013E08F011270091E706002309F045C106
:104BA0000091E606002351F4112309F43EC11BE0F5
:104BB0001093E70603950093E60637C1013039F4F8
:104BC0000091EE010130C9F0023059F0D5C0112337
:104BD00009F02BC11BE01093E70600270093E606BF
:104BE00024C11B3009F41AC11C3021F41127109381
:104BF000EE0114C110931C0411C1113031F40027CF
:104C00000093EE010E943E4A09C1123041F4F8942B
:104C10001091560104E0102710935701FFC0133084
:104C200041F4F8941091560108E0102710935701B1
:104C3000F5C0143041F4F8941091540100E81027A5
:104C400010935501EBC0153031F40E946B490FEF02
:104C500000934902E3C01730D1F4F89410E00E94A9
:104C6000E838302F0093DA062D912093DB061D9152
:104C70001093DC060D910093DD064D914093DE0606
:104C80004C914F7E4093DF060E94A339C7C0183075
:104C900051F5F89410E00E94E8380091E0060E9378
:104CA0000E7000933C041091FF0413FF00933D0429
:104CB00011960091E1060D930091E2060D9300918B
:104CC000E3060D930091E4060D930091E5060C9325
:104CD0000FEF0093490200930D0400270093770221
:104CE000009378029BC01930B1F4F89410E00E9450
:104CF000E8380093E0060D910093E1060D910093D2
:104D0000E2060D910093E3060D910093E4060D91E8
:104D10000093E50683C01B3089F4F89400910205E6
:104D2000102F0F77039505350CF00027F8940093AA
:104D300002050E9470390E94A33970C01A3041F4F4
:104D4000F8941091540108E010271093550166C0A3
:104D50001C3009F063C0F89400910205102F0F7702
:104D60000A9500230AF404E5F894009302050E94D2
:104D700070390E94A33952C0113011F4002735C098
:104D8000123011F405E031C0133011F40FE02DC0E2
:104D9000143011F404E129C0153011F409E125C0E3
:104DA000163011F40EE121C0173011F403E21DC0DA
:104DB000183011F408E219C0193011F40DE215C0D1
:104DC0001A3011F40AE011C01B3021F402E0009304
:104DD000EE0124C01C3011F501E00093EE01F894BF
:104DE0000E9470390E94A33919C0402F4B5F009375
:104DF000E1040E94F93817FD05C00091E104039514
:104E00000417A9F70FEF0093F50300930D04009327
:104E10004902002700937702009378020091E6068A
:104E200003950093E6060E94C73878940091FD032D
:104E3000002369F511271093FD030091FB0300FF88
:104E400026C01093FB031091020420910304021763
:104E500039F011271093040400930304102F09C0A4
:104E600020910404222329F4002312F013951395B2
:104E70001A951093020420914A02121719F02195F5
:104E8000121729F41127109302040093FD030091D7
:104E9000FE03002369F511271093FE030091FC0324
:104EA00000FF26C01093FC031091FF032091000423
:104EB000021739F011271093010400930004102FFA
:104EC00009C020910104222329F4002312F0139534
:104ED00013951A951093FF0320914A02121719F0A7
:104EE0002195121729F411271093FF030093FE0355
:104EF0000091F201002309F0C7C11091590116FD7C
:104F000005C002E00093F2010BE009C000914902E4
:104F1000002301F101E00093F20106E000C00093DC
:104F2000F70100270093F3010093F8010091EE01CF
:104F3000002371F0023061F000E20093A4030093BB
:104F4000A5030093A6030093A70300E20093D302F6
:104F50000C9439160091BB01002309F07BC000912D
:104F60005C0104FD2DC00FEF0093BB01F89400918C
:104F70005601037F0093560100935701009500935B
:104F80005C0110E60E940F38009154010F770093E6
:104F900054010093550100950093590110E30E94BC
:104FA0000F380FEF0093F8030093F90300270093E5
:104FB000ED010091FF04077F0093FF040C94391664
:104FC0000091BC01002309F009C000915C0100FDC3
:104FD0005AC30FEF0093BC010C9439160AE00093FA
:104FE0004A024091FE0340FF25C010E00E94E838CD
:104FF000102F0E70069547FF04C00A9532F407E0A3
:1050000004C0039508300CF00027000F00933C0407
:105010002091FF0423FF00933D04117F012B0E9389
:10502000F89400270093FE030FEF00934902789451
:105030000C94432B00915C0100FF0C94432B002740
:105040000093BC010093FF030093010401E000936F
:105050004A0219C30AE000934A020091F8030023B0
:1050600041F00091EA01002321F40093F8030E942B
:105070000F390091F903002341F00091E80100236A
:1050800021F40093F9030E942A391091FD0310FDC9
:105090001BC0F89400915C0102FD0AC00091D1028E
:1050A000002311F00C9439160FEF0093D10221C0A8
:1050B00003FD5CC00091D202002311F00C9439165C
:1050C0000FEF0093D20206C0F89429E01091FD037F
:1050D00017FF0FC00091E1040A9500230AF401E3D1
:1050E0000093E1040E94F93817FD12C02A9591F748
:1050F0003DC00091E1040395023309F400270093B9
:10510000E1040E94F93817FD03C02A9591F72EC0DB
:1051100010E00E94E8380E7000933C041091FF04E8
:1051200013FF00933D040E94F9380370109154015D
:105130001C7F002339F01260013021F01160033030
:1051400009F01D7F109355010E94C7380FEF00939F
:1051500049020093F50300930D04002700937702A2
:10516000009378020093FD030C9439164091FE03DE
:1051700040FF70C047FF1DC00091E1040023A1F073
:10518000053091F00A3081F00F3071F0043161F098
:10519000093151F00E3141F0033231F0083221F083
:1051A0000D3211F00A951CC000270093FE030C94E9
:1051B00039160091E1040430B9F30930A9F30E3037
:1051C00099F3033189F3083179F30D3169F3023230
:1051D00059F3073249F30C3239F3013329F30395BC
:1051E0000F930E94F9381F771C930F910093E104ED
:1051F0000E94F93810681C9310E00E94E8380E7085
:1052000000933C041091FF0413FF00933D040E949F
:10521000F9380370109154011C7F002339F012609B
:10522000013021F01160033009F01D7F109355010A
:105230000E94C7380FEF0093F50300930D0400930D
:105240004902002700937702009378020093FE033F
:105250000C943916112700915C0104FF0EC01093C5
:10526000BB010027009302040093FF030093040492
:105270000093010401E000934A02009149020023D7
:1052800009F45CC40C9439160091F501002311F067
:105290000C9439161091F701112339F11A951093D6
:1052A000F70111270091F8012091F301201729F44B
:1052B0002091F201213009F01FEF2091F1010E94AD
:1052C00034330091F801039516E02091F20121306A
:1052D00009F01BE0011709F400270093F8019093EF
:1052E000F6019093F5010C9439161091F2011230E9
:1052F00049F000270093F201009349020093F40162
:105300000C94391600914902002351F000270093B4
:1053100049020093F80106E00093F7010C94391656
:105320000091590106FDF5C0112700915C0100FFB5
:105330001FEF1093BC01112329F10091FE0300FF20
:1053400021C0112710937C0210931A0410931B04A0
:105350001093F8011091F101139507FD125022F0FE
:1053600012311CF0112701C011E11093F101002747
:105370000093FE0306E00093F3010BE00093F701B6
:105380000C9439160AE010917C02112321F00BE0F5
:105390000093F7010AE000934A022091FD0320FFE9
:1053A0002AC000270093FD030091BC01002331F0C7
:1053B00000270093BC010FEF0093BD010091F301A2
:1053C00027FD0A9507FD0AE00093F8010091F3011B
:1053D000200F0AE022F02B3000E009F0022F0093AA
:1053E000F30102E00093F701002700931A040093F1
:1053F0001B040C9439160091FE0300FD06C00091B9
:105400004902002311F40C94C12CF8E1E4EB109153
:10541000F10125E0129F22271091F3011630DCF1F3
:10542000100D4091F1014E3069F04F3059F01932B2
:1054300091F540913304442309F05DC04FEF409350
:10544000310429C040911B04040F43E522F0442796
:10545000043509F0402F40931B041FEF10931704ED
:105460001091F30116500091F1010E5025E0029FBA
:10547000100D1F7012952227B7E0A8E9A10FB21FE7
:1054800000911A04A00FB21FF7E0E2E5E40FF21F4B
:1054900004910C9330C0110F221F110F221FE10F36
:1054A000F21F15914591742F559164910E94CE3849
:1054B000802F4A9512F00695FCCF2091FE0305231C
:1054C00021F0061741F0020F09C022233AF06623AB
:1054D00029F0020F03C022230AF4020F7A951AF072
:1054E000000F550FFBCF50958523082BF8940C9394
:1054F0000E94C738789411271093FE031093490235
:1055000001E00093F7010091F3010093F8010C947E
:10551000CC2D002700937C021091BC01112329F0AF
:105520000093BC010FEF0093BD010091F301002334
:1055300062F001E00093F7010091F3010093F8019C
:105540000FEF0093F3010C9439160091F40100233E
:10555000A9F40FEF0093F4010091170400931804CD
:10556000F6E0E4E3B1E0A9EF0EE00E94C2380EE0FD
:105570000093F6010093F5010C943916002700936F
:10558000F4010093F20100931A0400931B040093AA
:1055900002040093FF0300930404009301040093AA
:1055A000170401E000934A0200910A0500FF0FC0B2
:1055B0000E7F00930A0500270093ED0618E7B4E07C
:1055C000ABE40D931A95E9F70FE70093EC0610E0B2
:1055D0000E94E8380E7000933C04102F0091FF04E5
:1055E00003FD1091E2041E7010933D040FEF009331
:1055F000490200930D0400937903009389020093FC
:10560000B0020091EE01002399F0023089F00DE420
:105610000093A403009115040093A50300911604C0
:105620000093A6030AE30093A70300E20093D302CA
:10563000009112050C7010911F04011711F40C94C5
:10564000391600931F0422271127002730911205D5
:105650003C7030931F0469F026E01DED00ED3430FE
:1056600041F02DE01BEB00EA303119F02BE117E798
:1056700000E4F89420932004109321040093220462
:1056800078940C9439160091EA01002309F08EC039
:105690000091ED0100FF23C000237AF4002700935E
:1056A000ED01F8940091FF04077F0093FF047894C4
:1056B0000E940F390E942A3979C000270093ED011A
:1056C000F8940091FF0408600093FF04789400911F
:1056D000E2040E7000933D040E94453967C0F894BF
:1056E0000091E90110915C01789400FF03C0002350
:1056F000C2F452C00091D202002309F057C013FD3A
:1057000055C00091FF04087009F450C01FEF1093BA
:10571000D2020E943F490E9445390FEF009349028F
:1057200045C00091EE0400680093EE0402E500938A
:10573000C9010AE30093CA01209170012093CB01B3
:10574000109171011093CC01009172010093CD0171
:10575000009173010093CE01009174010093CF0179
:1057600000917B010093D00100917C010093D10155
:1057700000917D010093D20100911305002341F0B7
:105780000E944B4A2093CA011093CB010093CC0195
:1057900005E10093EA0107C00E940F390091EE0471
:1057A0000F770093EE0400270093E9011091FF04A6
:1057B0000091E801002339F0187009F439C000277E
:1057C0000093EC01C4C0187009F421C00091D1020B
:1057D000002309F0BCC000270093EC0100915C019C
:1057E00002FDB5C01FEF1093D10210E00E94E8380F
:1057F000F8940093E2040D910093E3040D9100935B
:10580000E4040D910093E5040E944539A0C0109175
:10581000EE040091EB01002359F012F0116003C077
:105820000E942A391E7F1093EE0400270093EB019B
:1058300000270093EC0140915C0143FD41C04FEF14
:105840004093EC014091590147FD20C00091D002E6
:10585000002309F01BC00FEF0093D002F8940091D1
:10586000E6041091E704012B1091E804012B10913C
:10587000E904012B59F000270093E6040093E704A4
:105880000093E8040093E9040E94C7380091FE03E6
:1058900000FF16C0F8943091E6042091E7041091BF
:1058A000E8040091E9040E94E9323093E604209371
:1058B000E7041093E8040093E9040E94C738789441
:1058C00040915C0142FD5DC04FEF4093EC0140917F
:1058D000590147FD21C00091D002002309F01CC0EE
:1058E0000FEF0093D002F8940091EA041091EB04BA
:1058F000012B1091EC04012B1091ED04012B61F0B0
:1059000000270093EA040093EB040093EC04009357
:10591000ED040E94C73878940091FE0300FF31C067
:10592000F8943091EA042091EB041091EC0400917A
:10593000ED040E94E9320093ED041093EC042093EF
:10594000EB043093EA040E94C73878941AC000919F
:10595000FE0300FF16C0F89411E00E94E8380170C1
:10596000302F2D911D910C910E94E9320C931E93C2
:105970002E930E910E7F3170302B3C930E94C738CE
:10598000789410E00E94E838302F31702D911D91ED
:105990000D914091FF04487009F039C04091D40244
:1059A000442309F034C04091EC01442309F02FC096
:1059B0004091FE0340FF2BC0F8940E940833789476
:1059C00088277727662754E640911005442309F07D
:1059D0005AE040915C0141FD08C067E250E140910E
:1059E0001005442311F063E058EE4091FE03442378
:1059F00052F441E0509560957FEF8FEF540F40E0F7
:105A0000641F741F841F050F161F271F381F44278C
:105A10004093FE034091D402442309F08FC090913B
:105A2000FD0390FD25C04091140440FD0BC047FDCF
:105A300019C04091580142FD0CC0F8944460409355
:105A400058017894909114049E7F9093140491E0EF
:105A50000FC043FF02C00C94682DF8944860409337
:105A600058017894409114044F77409314049FEFA9
:105A700044274093FD03F8940E9408338827772732
:105A800066275AE040911005442309F051E0409107
:105A90005801427029F040915C01789441FD08C0A2
:105AA00063E058EE40911005442311F0662754E658
:105AB000992352F441E0509560957FEF8FEF540F9A
:105AC00040E0641F741F841F050F161F271F381F17
:105AD00070E060E057E24FE0401B510B620B730B2C
:105AE0006AF571E069EC53EC40E8401B510B620B26
:105AF000730B22F13F932F931F930F9310E00E949B
:105B0000E838302F31702D911D910D914F915F919B
:105B10006F917F91041739F4151729F4261719F49A
:105B2000371709F40BC0F8944E935E936E930E9161
:105B30000E7F702B7C930E94C738789410E00E94EF
:105B4000E838302F31702D911D910D914091FF0457
:105B5000487051F540915C0143FD26C07091E60408
:105B60006091E7045091E8044091E904040F151F87
:105B7000261F371F70E060E057E24FE0401B510BDB
:105B8000620B730B4AF471E069EC53EC40E8401B84
:105B9000510B620B730B42F410E00E94E838302F77
:105BA00031702D911D910D91882771E06BEA5EE3B4
:105BB0004FEF401B510B620B730B0AF08FEF80937A
:105BC00033040F931F932F933F93552745E00E9473
:105BD000453200911D04002329F000915308002351
:105BE00009F47FC00091E701002309F07AC0E4EDD9
:105BF000F1E0A0E7B1E089E077270091E30300231B
:105C000069F00091560106FD6CC00091420400232A
:105C100009F067C000270093E30375E10C9111912F
:105C2000011759F0813039F4003229F40091100540
:105C3000002309F402C01C9375E111968A9521F0A6
:105C4000843061F71696EACF00911005002319F40D
:105C500010E210937E01209131041127772319F46B
:105C6000222309F43EC01093310475E1009113051D
:105C7000002309F434C07BE1222311F077E21FEF07
:105C80001093320420917001109171017F930E9452
:105C90004B4A7F91209391011093920100939301BD
:105CA0000091720100939F01009173010093A00184
:105CB000009174010093A10100917C010093A30164
:105CC00000917D010093A40100917E010093A50144
:105CD00000911005002319F400E20093A5017093D0
:105CE000E7013F912F911F910F9174E063E35EE014
:105CF00048ED8091EF04882321F474E06CE25DE1CB
:105D000040E880913C04883011F18A3001F174E060
:105D100063E356E148EA8091EF04882321F474E0BC
:105D20006CE25AE34CEC80913C04803081F084308A
:105D300071F08C3061F074E063E357E048E08091EB
:105D4000EF04882321F474E06CE250E044E37F9395
:105D50006F935F934F93040F151F261F371F0093F8
:105D60006B0810936C0820936D0830936E08409177
:105D700070025AE0459FECE7F0E0E00DF11D772757
:105D8000659155914591332722271127002780914E
:105D90003C048830A1F08A3091F015910491843050
:105DA00071F08C3061F0803051F0009510952095A5
:105DB000309581E0080F80E0181F281F381F400F22
:105DC000511F621F731F0F911F912F913F914F938E
:105DD0005F936F937F93041B150B260B370B70910A
:105DE0000504609106045091070440910804041BC7
:105DF000150B260B370B00936F0810937008209338
:105E0000710830937208409171025AE0459FE0E5B5
:105E1000F2E0E00DF11D33272591159105917727CB
:105E200066275527442780913C048030D1F082308A
:105E3000C1F08830B1F08A30A1F05591449184309E
:105E400031F08C3021F0863061F08E3051F081E0FD
:105E50007095609550954095480F80E0581F681FD9
:105E6000781F040F151F261F371F7F916F915F91B9
:105E70004F91040F151F261F371F70910504609165
:105E800006045091070440910804040F151F261FB3
:105E9000371F7091090460910A0450910B044091DE
:105EA0000C04041B150B260B370B0093730810937F
:105EB0007408209375083093760880913C048830EC
:105EC00011F08A3069F40027112722273327009325
:105ED000830810938408209385083093860855C062
:105EE000409171025AE0459FE0E5F2E0E00DF11DBE
:105EF00033272591159105918030C9F08230B9F092
:105F00007727662755914491843019F08C3009F039
:105F10000AC081E07095609550954095480F80E0EB
:105F2000581F681F781F040F151F261F371F7091F9
:105F3000090460910A0450910B0440910C04041B65
:105F4000150B260B370B00938308109384082093BE
:105F5000850830938608772766275091170140916E
:105F6000180180913C04823061F0803071F481E04E
:105F70007095609550954095480F80E0581F681FB8
:105F8000781F040F151F261F371F009377081093E3
:105F900078082093790830937A0880913D044DE782
:105FA00030E023EA1FED03EB883029F14091290509
:105FB00030E023EA13ED0BEF8630E9F08E30D9F0B4
:105FC0004DE730E023EA1DE300E18A30A1F08030A4
:105FD00091F0823081F040912A0530E023EA1FEDF4
:105FE0000BE35091120557FF06C040912A0530E09F
:105FF00023EA0BE61BEE5527440F551F440F551F90
:10600000440F551F440F551F6627040F151F261FE9
:10601000361F00937B0810937C0820937D083093F3
:106020007E080E9405393E91317011962D911D9187
:106030000D914091560144FD14C04091FF044870F9
:1060400081F440915C0142FD0CC07091EA046091C2
:10605000EB045091EC044091ED04040F151F261F32
:10606000371F0F931F932F933F938091560186FD07
:1060700008C080914204882321F480911205807128
:1060800061F470917E0860917D0850917C08409188
:106090007B08040F151F261F371F00937F081093DE
:1060A00080082093810830938208882771E06FE48C
:1060B00051EB40E80E94B5380AF082608093C30239
:1060C00080911205807109F068C03F912F911F9156
:1060D0000F910F931F932F933F93882771E06BEAE3
:1060E0005EE34FEF401B510B620B730B0AF08FEF17
:1060F00090913304892B809333040E94D749F6F0A2
:1061000000913D0404302CF400913B0400FD0CC0D0
:1061100044C00A3009F441C00091560106FD3DC05B
:10612000009142040023C9F5002700937F080093E3
:10613000800800938108009382082FC010915601B7
:1061400016FD04C01091120515FD11C00027009323
:106150007F080093800800938108009382080093D1
:106160007B0800937C0800937D0800937E080091D3
:10617000E303002391F40091560106FD04C0009151
:106180004204002351F00091E203002331F407E1BF
:106190000093E2030FEF0093E3031091C10200911B
:1061A0002B05011779F00093C10215E0019F8001D2
:1061B00023E033270E94BF49009339041093380429
:1061C0004FEF14C0442736E0ABE6B8E0C7E8D8E0AC
:1061D00024E00D911991011709F041602A95C9F742
:1061E000440F3A95A9F7442309F48CC0F8944F93CF
:1061F00046FF13C000916B080093870810916C084C
:106200001093880820916D082093890830916E08BA
:1062100030938A0848E20E94FF314F914F9345FF27
:1062200013C000916F0800938B08109170081093B1
:106230008C082091710820938D083091720830935A
:106240008E0840E20E94FF314F914F9344FF13C0EC
:106250000091730800938F081091740810939008B0
:106260002091750820939108309176083093920818
:1062700048E10E94C8314F914F9343FF13C00091F2
:106280007708009393081091780810939408209150
:1062900079082093950830917A083093960840E366
:1062A0000E94C8314F914F9342FF13C000917B0869
:1062B0000093970810917C081093980820917D080E
:1062C0002093990830917E0830939A0840E10E940B
:1062D000C8314F9141FF13C000917F0800939B0884
:1062E0001091800810939C082091810820939D08AC
:1062F0003091820830939E0848E30E94C8310E9482
:10630000413278943F912F911F910F914091BB01A1
:106310004423E1F54091BC014423C1F54091FF04C1
:10632000487021F440915C0142FD30C0552745E0A2
:106330000E9445320091E801002341F5E4EDF1E0CF
:10634000A3EBB1E088E077270C911191011711F0D0
:106350001C9375E111968A9509F0F6CF7093E801C8
:1063600008E50093B1010AE30093B201009113051F
:10637000002361F02091B3011091B4010E944B4AB7
:106380002093B2011093B3010093B4010C94391619
:106390004F93332352F4009510952095309541E0AA
:1063A000040F40E0141F241F341F67E15BED41E937
:1063B00070913904470F70913804571F70E0671FC0
:1063C0000E9440352F912F9301E00E9444380091A4
:1063D0000E042F912F930E94443800910F042F91A7
:1063E0002F930E944438009110042F912F930E9404
:1063F0004438009111042F910E94443808954F931E
:10640000332352F4009510952095309541E0040F08
:1064100040E0141F241F341F6EE050E54AE87091DD
:106420002B05470F70E0571F671F0E9440352F91C3
:106430002F9300910E0414E00E948B3800910F04FA
:106440002F912F9315E00E948B38009110042F910B
:106450002F9316E00E948B38009111042F912F93F7
:1064600017E00E948B38009112042F912F9318E0AF
:106470000E948B38009113042F9119E00E948B38F1
:1064800008952F9A00002F9808955F934F9340E24C
:1064900033235AF4309520951095009541E0040F70
:1064A00040E0141F241F341F4DE24F93442755270B
:1064B000662778E183E090E3000F111F221F331F4E
:1064C000441F551F661F7A9589F160935101680F2B
:1064D00063FF6091510160935101690F67FF609103
:1064E000510150935101580F53FF50915101509356
:1064F0005101590F57FF5091510140935101480FDD
:1065000043FF4091510140935101490F47FF409192
:10651000510130935101380F33FF309151013093C5
:106520005101390F37FF30915101C6CF1F910F91A3
:106530002EE2A3EDB1E01D93762F72957F7070630C
:106540007D93013009F42D936F7060636D93023079
:1065500009F42D93752F72957F7070637D930330CE
:1065600009F42D935F7050635D93043009F42D930B
:10657000742F72957F7070637D93053009F42D93AD
:106580004F7040634D93063009F42D93732F72952D
:106590007F7070637D93073009F42D933F703063F3
:1065A0003D93083009F42D935F91552309F0089528
:1065B000199721E03D91303349F4021739F01297D1
:1065C00030E23D931D9323952930A1F712971C9338
:1065D00008954091D402442309F008950E9408339D
:1065E0007727662755274AE080915C0181FD02C02C
:1065F00053E048EE8091FE0388232AF4041B150B18
:10660000260B370B0895040F151F261F371F0895FB
:106610000F9300915C0101FD25C0009112050370EC
:1066200059F00130B1F0023069F005E70093EA0655
:1066300000E30093EB0613C000270093EA060093E3
:10664000EB060DC00AE30093EA0608E90093EB06A7
:1066500006C003E10093EA0608E80093EB06002772
:106660000093D4020F910895422FE8E2F7E144230A
:1066700009F445C0EEE3F7E1413009F440C0E4E538
:10668000F7E14230E1F1EAE6F7E14330C1F1E0E859
:10669000F7E14430A1F1E6E9F7E1453081F1ECEAB8
:1066A000F7E1463061F1E2ECF7E1473041F1E8ED26
:1066B000F7E1483021F1EEEEF7E1493001F1E4E095
:1066C000F8E14A30E1F0EAE1F8E14B30C1F0E0E313
:1066D000F8E14C30A1F0E6E4F8E14D3081F0ECE572
:1066E000F8E14E3061F0E2E7F8E14F3041F0E8E8E0
:1066F000F8E1403121F0EEE9F8E1413101F00430F8
:1067000039F420910005287019F0F7E1ECE10DC093
:10671000000F2227E00FF21F069535912491330FC9
:10672000221FF9E0E6E8E30FF21FD1E0C9EF26E00F
:10673000922F359139932A95E1F72FE1299328E299
:10674000299327E6299321E0299329939B5F11231D
:1067500039F02FE1299322E7299321E029939D5FC6
:106760002591222349F435913093480125912993AD
:1067700093953A95D9F72591043029F43091000585
:10678000387009F0B4C0B8E1A4EB35E0439F06309F
:106790000CF0000D4427000F441F000F441FA00FF2
:1067A000B41F35913323DAF1FF93EF93FD01449148
:1067B000EF91FF9146379CF046574F704295B7E0F6
:1067C000A8E9A40F40E0B41F3CE02D91222329F05A
:1067D000299393953A95C9F78AC020E284C044274B
:1067E0004093FA031F93FF93EF93FD011591459199
:1067F000559164910E94CE384A9512F00695FCCFCF
:106800000523039FEF91FF911F91E00DF11D25914D
:10681000222321F0299393953A95C9F768C04FEF49
:106820005527222312F444275FEF40937C025093B4
:10683000FA033195432F1F939F93CF93DF93FD016D
:10684000BB27A491552339F01A2F0E94CE38332745
:106850002227112705C0B1E0332722271D910C9173
:1068600055270E944532DF91CF919F911F91009152
:10687000480131E1301B313079F1323041F13330B0
:1068800009F13430D1F0353099F0363061F03730DD
:1068900029F00091D401099393953A950091D5017F
:1068A000099393953A950091D601099393953A955A
:1068B0000091D701099393953A950091D8010993D6
:1068C00093953A950091D901099393953A95009142
:1068D000DA01099393953A950091DB010993939519
:1068E0003A9529F020E2299393953A95E1F71123FF
:1068F00039F00FE1099302E7099300E009939D5FE6
:106900000895F8943091530130653BB93FEF37B9A2
:1069100030915B0138B9439A449829980E942E35EA
:106920000E942E35299A0E942E35449A29980E9459
:106930002E350E942E35299A0E942E350E942E3522
:10694000439829980E942E350E942E35299A0E943C
:106950002E350E942E350C3911F00E3961F40E944B
:10696000E134012F0E94E134022F0E94E13400271C
:106970000E94E13408C00E94E134012F0E94E134FA
:10698000022F0E94E1340E942E350E942E35449A37
:1069900029980E942E350E942E35299A0E942E3564
:1069A000439A29980E942E350E942E35299A0E94DA
:1069B0002E35449829980E942E350E942E35299A0A
:1069C000089538E0449A000F08F4449829980E94EA
:1069D0002E350E942E35299A439A29980E942E35E9
:1069E0000E942E35299A0E942E35439829980E949C
:1069F0002E350E942E35299A0E942E350E942E3562
:106A00003A9501F7449829980E942E350E942E3518
:106A1000299A439A29980E942E350E942E35299A48
:106A2000C0915301C062CBB9CC27C7B929980E9445
:106A30002E350E942E35C6B1299AC0915301C065EA
:106A4000CBB9CFEFC7B9C0915B01C8B943982998BA
:106A50000E942E350E942E35299A089500000000CC
:106A60000895F999FECFB2BDA1BDF89A00B5089579
:106A7000F999FECFB2BDA1BD00BDFA9AF99A089569
:106A8000772770930E0470930F0470931004709323
:106A90001104709312047093130440FD0E94573543
:106AA00066955795479573957631B9F70895882778
:106AB0009927A32FB22FC12FD02FE72FEE2341F01C
:106AC000DD0FCC1FBB1FAA1F991F881FEA95F6CFA9
:106AD000E0911304DE0FD0931304E0911204CE1F53
:106AE000C0931204E0911104BE1FB0931104E09111
:106AF0001004AE1FA0931004E0910F049E1F90930A
:106B00000F04E0910E048E1F80930E0408950091EF
:106B1000FF04007841F500270093500800936901B5
:106B20000093E7010093EA010093E8010093F50167
:106B30000093E9020093EA020093B9030093D302A1
:106B40000093BA030093E2030093F4030093F60367
:106B500000937803009337040093490400937F0265
:106B600000938002089501E010906701011509F477
:106B700092C10395011509F409C20395011509F4A1
:106B8000CDC00395011509F4E6C00395011509F47C
:106B9000F0C00395011509F4FAC00395011509F435
:106BA00006C10395011509F410C10395011509F4F7
:106BB0001AC10395011509F424C10395011509F4BF
:106BC0002EC10395011509F438C10395011509F487
:106BD00042C10395011509F44CC10395011509F44F
:106BE000B9C10395011509F464C10395011509F4B0
:106BF0009BC10395011509F46AC10395011509F4B8
:106C000084C10395011509F4D0C101E0209050081A
:106C1000222009F040C100911D04002361F0009181
:106C20005308002309F4D7C100915108109152086C
:106C3000012B09F0D0C102E020906901222009F067
:106C4000A5C103952090E701222009F067C00395B4
:106C50002090EA01222009F07EC003952090E801EF
:106C6000222009F086C003952090F501222009F02A
:106C70008EC003952090E902222009F098C0039568
:106C80002090EA02222009F0A0C003952090B903C9
:106C9000222009F0A8C003952090D302222009F0F9
:106CA000B0C003952090BA03222009F0B8C0039524
:106CB0002090E203222009F0C0C003952090F40345
:106CC000222009F0C8C0039520907803222009F003
:106CD000D0C003952090F603222009F03BC1039514
:106CE00020903704222009F0E4C003952090490445
:106CF000222009F019C1039520907F02222009F07B
:106D0000E6C0039520908002222009F0FEC0039582
:106D100020904404222009F048C15DC1009367011E
:106D200004E1EAE6F1E010911305112359F0EBE8D4
:106D3000F1E00AE110913204112321F01CE0010F6F
:106D4000E11BF0402090E7012A942092E70102190C
:106D5000102E442444C1009367012090EA012A9434
:106D60002092EA0104E10219102EEEEBF1E0442436
:106D700036C1009367012090E8012A942092E8012F
:106D800004E10219102EE6EAF1E0442428C1009340
:106D900067012090F5012A942092F5010091F601F7
:106DA0000A950219102EE9EFF1E0442418C100936E
:106DB00067012090E9022A942092E90200E1021979
:106DC000102EE8EDF2E044240AC100936701209000
:106DD000EA022A942092EA020FE60219102EECEE43
:106DE000F2E04424FCC0009367012090B9032A9488
:106DF0002092B90305E10219102EEBE7F3E04424D9
:106E0000EEC0009367012090D3022A942092D3020F
:106E10000FE10219102EE9E9F3E04424E0C00093E9
:106E200067012090BA032A942092BA030EE0021957
:106E3000102EECEBF3E04424D2C0009367012090C5
:106E4000E2032A942092E20306E10219102EEBECF1
:106E5000F3E04424C4C0009367012090F4032A9413
:106E60002092F4030FE00219102EE4EEF3E0442424
:106E7000B6C01091590116FFAEC000936701209073
:106E800078032A94209278030BE10219102EECE586
:106E9000F3E04424A4C000936701209050082A9492
:106EA0002092500807E10219102EE8E3F8E044248C
:106EB00096C000936701209037042A9420923704EB
:106EC00006E10219102EE4E5F8E0442488C000939E
:106ED0006701112720907F0227FE02C021941FEF37
:106EE0002A9420927F0209E10219102E043144F005
:106EF000112331F013941394139413941394139453
:106F0000E6E0F7E0442440946AC0009367012090D3
:106F100080022A94209280020BE10219102EE6E2F0
:106F2000F7E0442440945BC000936701209049043B
:106F30002A94209249040BE00219102E0B3029F4F8
:106F40000091480405FD01C01394ECEAF6E04424E6
:106F5000409445C0009367012090F6032A94209244
:106F6000F60302E00219102E00912F05000F000F0A
:106F7000E8EBF5E0E00F00E0F01F0091F7030023DD
:106F800011F4E4EBF5E04424409429C00093670138
:106F9000209069012A942092690103E10219102EC0
:106FA000E0EAF5E0442440941AC000936701209081
:106FB00044042A94209244040BE00219102E0B3052
:106FC00029F40091450405FF01C01394E6E2F6E0C0
:106FD0004424409404C0222420927D0208950AE0B3
:106FE00000937E0200916701222009F4002700939C
:106FF00067012224E10DF21D008040FCC895002DA0
:107000001FEF17B918B90E942E350E942E3508B906
:107010000E942E352E980E942E352E9A0895F894AF
:107020002FEF103328F42FEF28B9222727B904C0F7
:1070300028B927B9000008B900915301012B0BB9F9
:1070400000000000000029980E942E350E942E3575
:1070500006B1299A08950F931F93F89400915A014D
:107060000F7700935A0110E40E940F381F910F917F
:107070000E940F3800915A01006800935A0110E4F1
:107080000E940F38789408950F932F93F8940091ED
:107090005A01022B10E40E940F382F910F9108B96A
:1070A0000E942E350E942E35289A0E942E350E946D
:1070B0002E3528980E942E350E942E35089508B945
:1070C0000E942E350E942E35289AAA27B4E31197E4
:1070D00011F01B99FCCF2898AA27B4E3119711F05F
:1070E0001B9BFCCF0E942E350E942E350895289AB6
:1070F000AA27B4E3119711F01B99FCCF06B1289889
:10710000AA27B4E3119711F01B9BFCCF0E942E35E8
:107110000E942E3508950F931F932F93F89400919A
:107120005A01022B10E40E940F382F911F910F91EA
:10713000009508B91F9310952C9814FD2C9A2D9842
:1071400015FD2D9A1F9112951095107F00915301F6
:10715000012B0BB90E942E350E942E35289A0E94D1
:107160002E350E942E3528980895002E041B002DE0
:10717000012E150B102D022E260B202D032E370B62
:10718000302D089515911D930A95E1F7089503E1B7
:107190000093E80608E80093E9060895B4E0A1EE3C
:1071A000112342F0133311F01D3369F40091C20230
:1071B000100F09C0B5E0A6E32091E10406E0029FAC
:1071C000A00DB11D1095A10F10E0B11F0C910895F5
:1071D000112329F0B4E0A1EE012E112406C0B5E080
:1071E000A6E31091E10406E0019FA00DB11D0D91F1
:1071F0000895B5E0A6E30091E10416E0109FA00D0C
:10720000B11D14960D911C91089510E00091FF049A
:10721000087009F011E00E94E8380E70089500E24D
:107220000093C9010093CA010093CB010093CC01E4
:107230000093CD010093CE010093CF010093D001C4
:107240000093D1010093D201F89405E10093EA0183
:107250007894089500E20093B1010093B201009385
:10726000B3010093B4010093B5010093B6010093FC
:10727000B7010093B8010093B9010093BA01F894E3
:1072800005E10093E80178940895E0E5F6E00091C7
:10729000E2040695077018E0109FE00DF11D0591BE
:1072A0000093C90105910093CA0105910093CB0198
:1072B00005910093CC0105910093CD0105910093B8
:1072C000CE0105910093CF0105910093D00100E21A
:1072D0000093D1010093D20105E10093EA010895E2
:1072E000B1E0AAEF00910205102F0F7705351CF0D1
:1072F00010781093020516E0019FA00DB11D0E94A9
:107300003135302F31700093DA0611960E943135F5
:10731000202F2093DB0611960E943135102F1093F9
:10732000DC0611960E9431350093DD060F9311960D
:107330000E9431350093DE0611960E94313500938C
:10734000DF060F91089545E00E9445320091D30277
:10735000002309F008950DE40093A4030AE30093C9
:10736000A7030091D4010093A8030091D5010093D5
:10737000A9030091D6010093AA030091D7010093BD
:10738000AB030091D8010093AC030091D9010093A5
:10739000AD030091DA010093AE030091DB0100938D
:1073A000AF0300E20093B00348E033272227112700
:1073B000009102050E9445320091DA010093A50375
:1073C000009315040091DB010093A60300931604BB
:1073D000E0E5F6E00091DA060E70069518E0109FE1
:1073E000E00DF11D05910093B10305910093B203E7
:1073F00005910093B30305910093B40305910093A5
:10740000B50305910093B60305910093B703059169
:107410000093B80300E20093D3020895002700937D
:107420004B020091F406002309F4089500914607E9
:10743000002309F00895F7E0EAECB6E0A6EF2FE6A6
:107440001D911F7D05910117C1F4009348071C9100
:107450001F7D04910117A9F4009349071196112784
:107460000C910B3309F41FEF109382023196C591F2
:10747000D491FE01D7E0CAE4099433962A9511F716
:1074800004C0119733962A95D9F6D7E0C8E40FE3E4
:1074900009930FEF0093820202E011C033272227E5
:1074A00011275FEF48E00E9445320091D90109930E
:1074B0000091DA0109930091DB01099306E01BE3D7
:1074C000188300934707009346070091C1000062AC
:1074D0000093C10000270093F4060091820200FF90
:1074E0000E94C7381FEF10934B020895112371F0CB
:1074F00010E30091540105FD11E31993199310E372
:107500000091480407FD11E319931AC00D910993E6
:107510000E94DC4802300AF0B8CF302F0E94DC48CD
:1075200002300AF0B2CF10915401332329F415FD33
:107530001F7D1093550104C015FF10621093550173
:1075400006E0BDCF112341F00091900240919202DC
:1075500040FD00919102A2CF63E00E94A5480AF489
:1075600094CF222309F091CF109391020FEF009353
:10757000920206E0A4CF112341F0009194024091C1
:10758000960240FD0091950289CF63E00E94A548D4
:107590000AF47BCF222309F078CF109395020FEFE6
:1075A0000093960206E08BCF112349F010E300917F
:1075B0001205007409F011E3199304E080CF0E94D2
:1075C000DC4802300AF061CFF894109112051F7B5D
:1075D00000FD006400931205789404E070CF11233D
:1075E00069F00E94053913960C910870069506956E
:1075F00006950395005D099304E061CF0E94DC4885
:10760000013019F0023009F040CF0A95000F000F49
:10761000000F0F93F8940E94053913960C91077F81
:107620001F91012B0C9378940FEF00934B0204E011
:1076300046CF112361F00E94F93800710695069536
:10764000069506950395005D099304E038CF0E94E6
:10765000DC48013019F0023009F017CF0A95000F0D
:10766000000F000F000F0F93F8940E94F9380E914D
:107670000F7E1F91012B0C9378940FEF00934B0218
:1076800004E01DCF112349F010E30091FF040170C5
:1076900009F011E3199304E012CF0E94DC48023094
:1076A0000AF0F3CEF8941091FF041E7F012B009393
:1076B000FF04789404E003CF112349F010E3009114
:1076C0005D01007809F011E3199304E0F8CE0E94FF
:1076D000DC4802300AF0D9CEF8940F930E94F938B2
:1076E0000F7D1F91110F110F110F110F110F012B92
:1076F0000E93789404E0E3CE112339F0009108054D
:1077000010E3010F099304E0DACE0E94DC48083050
:107710000AF0BBCEF89400930805789404E0CFCE2D
:10772000112349F010E300911205007109F011E3F3
:10773000199304E0C4CE0E94DC4802300AF0A5CEC2
:10774000F894109112051F7E002311F000E1102B18
:1077500010931205789404E0B2CE0027112349F06B
:1077600000910E059BCE03E0112319F000910F0547
:1077700095CE0F9363E00E94A5480F910AF485CE41
:10778000222309F082CE202F06E0222319F4109341
:107790000E0595CE213019F410930E0590CE2230AF
:1077A00019F410930E058BCE10930F0588CEF5E0DB
:1077B000E4E133270091C202E00FF31F112311F01F
:1077C00000816CCE63E00E94A5480AF45ECE2223BD
:1077D00009F05BCE108306E072CEF5E0EEE13327D0
:1077E0000091C202E00FF31F112311F0008156CE69
:1077F00063E00E94A5480AF448CE222309F045CE52
:10780000108306E05CCE112319F000912A0546CEC4
:1078100063E00E94A5480AF438CE222309F035CE51
:1078200010932A0506E04BCE112319F0009129058B
:1078300035CE63E00E94A5480AF427CE222309F042
:1078400024CE1093290506E03ACE112319F00091B9
:107850002C0524CE63E00E94A5480AF416CE22230C
:1078600009F013CE10932C0506E029CE112331F137
:1078700000910C053327222711275FEF48E00E9473
:1078800045320091D90109930091DA0109930091E1
:10789000DB01099300910D053327222711275FEFA4
:1078A00048E00E9445320091D90109930091DA0124
:1078B00009930091DB01099309E001CE63E00E9486
:1078C000A5480AF4E2CD222309F0DFCD10930C0580
:1078D00063E00E94A5480AF4D8CD222309F0D5CD53
:1078E00010930D0509E0EBCD112349F010E3009151
:1078F0001205007209F011E3199304E0E0CD0E9433
:10790000DC4802300AF0C1CDF894109112051F7DB9
:10791000002309F0106210931205789404E0CFCD93
:10792000112319F000912805B9CD63E00E94A54804
:107930000AF4ABCD222309F0A8CD1093280506E068
:10794000BECD112319F000913505A8CD63E00E944A
:10795000A5480AF49ACD222309F097CD1093350556
:1079600006E0ADCD112319F000912B0597CD63E012
:107970000E94A5480AF489CD222309F086CD1093F0
:107980002B0506E09CCD00911404006800931404BC
:1079900003E095CD112319F00091FD047FCD63E044
:1079A0000E94A5480AF471CD222309F06ECD1093F0
:1079B000FD0406E084CD112349F010E30091110588
:1079C000007409F011E3199304E079CD0E94DC48BA
:1079D00002300AF05ACDF8941127002309F010E480
:1079E00010931105789404E06ACD112339F010E367
:1079F0000091540103FD11E3199318C00E94DC4863
:107A000012F0023014F00C94453A10915401002306
:107A100019F413FF0BC002C013FD08C0F8941091B5
:107A2000540108E0102710935501789404E00C9459
:107A30005F3A112339F010E300912D05010F0993EE
:107A400004E03DCD0E94DC4803300AF01ECDF894DE
:107A500000932D05789404E032CD112349F010E312
:107A600000911205007809F011E3199304E027CD85
:107A70000E94DC4802300AF008CDF89410911205FB
:107A80001F77002309F0106810931205789404E022
:107A900016CD0091140401600093140403E00FCD8F
:107AA000112321F010E00E94E04809CD10E00E946F
:107AB00009490AF4EACC03CD112321F011E00E9418
:107AC000E048FDCC11E00E9409490AF4DECCF7CC75
:107AD000112349F010E300910005087009F011E34B
:107AE000199304E0ECCC0E94DC4802300AF0CDCCC3
:107AF000F89410910005177F002309F01860109387
:107B000000050FEF00934B02789404E0D8CC00916D
:107B10008308402F10918408412B20918508422B27
:107B200030918608432B31F445E335E320E310E33D
:107B300000E30EC0552748E00E9445324091D7012E
:107B40003091D8012091D9011091DA010091DB0127
:107B50004993399329931993099308E0B0CC1123E1
:107B6000B1F0009109050F71002311F014E0010F2D
:107B70003327222711275FEF48E00E94453200910A
:107B8000DA0109930091DB01099305E098CC62E0EA
:107B90000E94A5480AF479CC222309F076CC15314D
:107BA0000AF073CC112321F0145009F00AF411E00B
:107BB000F894009109050078102B1093090578942A
:107BC00005E07DCC112339F00091EF0410E3010FA3
:107BD000099304E074CC0E94DC4802300AF055CCD2
:107BE0000093EF0404E06BCC112321F024E0F4E0D7
:107BF000E4EF0FC00C91005302300AF046CCF4E0E1
:107C0000E4EF442734E019C0112379F024E0F4E0D4
:107C1000E0EF019110E30A3012F011E60A50010F73
:107C200009932A95B1F707E04ACC0C91003309F08B
:107C30002CCCF4E0E0EF4FEF34E00E94DC4844232A
:107C400089F40A308AF0102F10620AE0113361F0D3
:107C50000395123349F00395133331F00395143330
:107C600019F013CC0930EAF701933A9531F707E0A0
:107C700026CC112321F000E3099304E020CC0E94DC
:107C8000DC4810E3002369F0013019F0023021F0E4
:107C9000FCCB0E943F4905C00E946B490FEF009347
:107CA0004B02F8940091540107FF03C00F77009333
:107CB0005501789404E003CC112349F000E31091BE
:107CC000FF04187009F001E3099304E0F8CB0E9467
:107CD000DC4810E3002361F0013009F0D6CBF894C2
:107CE0000091540107FD0DC000680093550109C0C3
:107CF000F8940091540107FF04C00F7700935501D9
:107D00007894789404E0DBCB112349F010E30091E0
:107D10005C01027009F011E3199304E0D0CB0E94DA
:107D2000DC4802300AF0B1CBF894109156011D7F67
:107D3000000F00950270012B00935701789404E026
:107D4000BECB00913A04002309F04AC0112321F16F
:107D500010E00E94E838007340913C0444305CF02D
:107D60004C304CF410E3199319931993002309F440
:107D700011E3199374C0003224F031F010E324E3CE
:107D800005C012E324E302C011E328E31993299309
:107D900010E31993199363C064E00E94A5480AF4A4
:107DA00074CB40913C0444305CF04C304CF41230C5
:107DB0000CF06BCB109511701295212F3FEC44C045
:107DC00038EE43E01317240700E338F030ED47E0C6
:107DD0001317240700E208F000E1202F3FEC34C025
:107DE0001123A9F010E00E94E83810E307FD11E329
:107DF000199310E306FD11E3199310E305FD11E358
:107E0000199310E304FD11E3199307E058CB0E9486
:107E1000DC4802300CF039CB202F220F0E94DC48C6
:107E200002300CF032CB202B220F0E94DC480230B3
:107E30000CF02BCB202B220F0E94DC4802300CF0E0
:107E400024CB202B22953FE010E00E94E83803234A
:107E5000022B0E930FEF0093790300930D0407E0BC
:107E60002ECB112369F010E00E94E838007C0295C7
:107E700006950695039510E3010F099304E01FCBC7
:107E80000E94DC48002311F005300CF0FECA0A9570
:107E9000000F000F0295202F10E00E94E8380F73AA
:107EA000022B0E930FEF0093790300930D0404E06F
:107EB00006CB112359F010E00E94E83800730295B8
:107EC000039510E3010F099304E0F9CA0E94DC480E
:107ED000002311F005300CF0D8CA0A950295202F26
:107EE00010E00E94E8380F7C022B0E930FEF0093F6
:107EF000790300930D0404E0E2CA112359F000E372
:107F0000099309930E94F93810761295106319931A
:107F100006E0D5CA0E94DC480E94DC480E94DC488A
:107F2000002339F0023029F0043019F0063009F04E
:107F3000ACCA02950F930E94F9381F790F91012B5B
:107F40000C930FEF00934B0206E0B9CA112349F0DE
:107F500010E300912E05002309F011E3199304E0CA
:107F6000AECA0E94DC4802300AF08FCAF89400932F
:107F70002E05789404E0A3CA07E3099301E309936B
:107F800000E3099306E09BCA10E00E94E0480091DC
:107F90003A040023E1F00091ED041091EC042091EB
:107FA000EB043091EA045FEF48E00E944532009113
:107FB000D30109930091D80109930091D901099344
:107FC0000091DA0109930091DB01099306C000E2F8
:107FD000099309930993099309930091E904109176
:107FE000E8042091E7043091E6045FEF48E00E9446
:107FF00045320091D30109930091D8010993009172
:10800000D90109930091DA0109930091DB010993E9
:1080100010E30091EE0407FD11E3199310E30091C2
:10802000EE0400FD11E3199310E219930091150479
:1080300000630993009116040063099310E3009113
:10804000560106FD11E300914204002309F011E3FB
:1080500019930E94824A199310E30091300400FDA5
:1080600012E3199310E300912F0400FD11E319931B
:1080700010E30091FF0403FD11E3199300E309935A
:108080000993099300E2099306E219CA112341F109
:108090003091050420910604109107040091080412
:1080A00040913A04442341F03091090420910A049C
:1080B00010910B0400910C045FEF48E00E944532E0
:1080C0000091D30109930091D80109930091D9013E
:1080D00009930091DA0109930091DB0109933DC0F6
:1080E0000D91003229F00B3219F00D3209F0CDC993
:1080F00009930F9364E00E94A54812F40F91C5C93B
:10810000012F122F083E43E0140718F431E022E358
:108110000FC0003D47E0140718F432E024E608C021
:10812000083843E1140710F00F91AFC933E02AEF8C
:1081300030683093790233270E94BF491F911D3266
:1081400009F4019510913A0410FF0093770210FD95
:10815000009378020FEF00930D0408E0B0C91123DB
:1081600061F010E3009100050073069506950695F1
:108170000695010F099304E0A2C90E94DC48033070
:108180000AF083C9F894000F000F000F000F109140
:1081900000051F7C102B10930005789404E08FC914
:1081A000112349F000911A011091A502112311F039
:1081B0000091A40273C963E00E94A5480AF465C94E
:1081C000222309F062C910340AF05FC915300AF49D
:1081D0005CC91093A4020FEF0093A50206E06FC9DB
:1081E000112369F010E300914204002321F400916F
:1081F0005601067009F011E3199304E060C90D916E
:108200000993F7E0E8E91CE022270D9109930C336C
:1082100009F42FEF01931A95C1F734961CE00D91E4
:10822000099301931A95D9F701E0222309F400E894
:1082300000931C040FEF009318040CE140C91123B4
:1082400041F010E3009100050770010F099304E06D
:1082500036C90E94DC4805300AF017C9F89410911D
:108260000005187F102B10930005789404E027C9AF
:10827000112339F010E30091D40200FD11E31993AA
:1082800010C00E94DC481127002321F01FEF0130AD
:1082900009F0FBC81093D402109510FF13951093AA
:1082A000BB0304E00CC9112341F010E30091120557
:1082B0000370010F099304E002C90E94DC480430F6
:1082C0000AF0E3C8F894109112051C7F102B10934C
:1082D0001205789404E0F3C8112349F010E30091EB
:1082E0003105002309F011E3199304E0E8C80E9466
:1082F000DC4802300AF0C9C8F894889407950795BD
:1083000000933105789404E0DAC8112351F000E2BB
:1083100009930091150400630993009116040993D1
:1083200019C00D9109930D910F930C910F93119713
:1083300062E00E94A5480AF402C015351CF00F91B6
:108340000F9108C00F91009316040F91009315042C
:108350001093020506E0B3C8112321F00E94824A5F
:1083600019932DC00C91099322270333B1F0239563
:10837000073399F02395023381F02395013369F097
:108380002395053351F02395043339F023950633B3
:1083900021F02395093309F078C8220F10E00E94DC
:1083A000E838017F022B0E930E7000933C0410916D
:1083B000FF0413FF00933D040FEF00934B0204E012
:1083C0007EC8112341F00091970210919A0210FD8E
:1083D0000091990263C863E00E94A5480AF455C859
:1083E000222309F052C8109399020FEF00939A02CA
:1083F00006E065C80D9109930D91099362E00E9412
:10840000A54815350AF041C8B1E0AAEF06E0019F82
:10841000A00DB11D0E9431350F700F9301700F93A5
:1084200011960E9431350F9311960E9431350F93AA
:1084300011960E9431351F912F913F915FEF48E0D7
:108440000E94453200E30993099309930091D401F6
:1084500009930091D50109930091D60109930091E8
:10846000D70109930091D80109930091D90109938B
:108470000091DA0109930091DB0109930F910695B0
:108480000E94864A199300E309930993099309937B
:1084900000E2099308E113C80D9109930D91099326
:1084A00062E00E94A548153512F00C94453A1F93DE
:1084B00068E00E94A5485F9112F40C94453A0C9133
:1084C000005312F40C94453A0A3012F00C94453AD9
:1084D00009930E949D4A660FB1E0AAEF06E0059F4E
:1084E000A00DB11D042F0170062B0E943835119686
:1084F000032F0E9438351196022F0E9438351196AD
:10850000012F0E94383500E30993099309930993D9
:1085100008E10C945F3A112339F010E30091540103
:1085200002FD11E3199318C00E94DC4812F00230DA
:1085300014F00C94453A10915401002319F412FFE1
:108540000BC002C012FD08C0F8941091540104E061
:10855000102710935501789404E00C945F3A11238E
:1085600039F00E94F93820E314FD21E3299312C069
:108570000E94DC483327002329F030E1013011F05C
:108580000C94453A0E94F9381F7E132B1C930FEF71
:1085900000934B0204E00C945F3A112349F00091E0
:1085A00085021091880210FD009187020C944E3ACA
:1085B00063E00E94A54812F40C94453A222311F07E
:1085C0000C94453A109387020FEF0093880206E05F
:1085D0000C945F3A112379F00E94F9381C70012F36
:1085E00010E3002321F011E3043009F012E31993A2
:1085F00004E00C945F3A0E94DC48033012F00C94C3
:10860000453AF8940F930E94F938137F0F91000FA9
:10861000000F102B1C93789404E00C945F3A112304
:1086200079F020E3009154010370002320E331F03E
:10863000023021F021E3013009F022E3299319C02F
:108640002C9129933091540130FD3D7F32702033BD
:1086500041F031E0213329F033E0223311F00C9462
:10866000453AF894009155010C7F032B0093550176
:10867000789404E00C945F3A112309F111270091DA
:1086800089022091FF042670243031F0263021F039
:1086900033272AE00E94BF493327222711275FEFA3
:1086A00048E00E9445320091D90109930091DA0116
:1086B00009930091DB01099306E00C945F3A63E0B3
:1086C0000E94A54812F40C94453A4091FF0446706C
:1086D000443051F0463041F01C3010F00C94453AD3
:1086E0000AE0019F102D04C0113810F00C94453A97
:1086F00010938C020FEF00938D0206E00C945F3A0A
:10870000112359F010E3009112050C70069506959F
:10871000010F099304E00C945F3A0E94DC48043096
:1087200012F00C94453AF89410911205137F000F43
:10873000000F102B10931205789404E00C945F3A0C
:10874000112349F000919F021091A20210FD0091A7
:10875000A1020C944E3A63E00E94A54812F40C94D6
:10876000453A222311F00C94453A1093A1020FEFE1
:108770000093A20206E00C945F3A112351F010E33B
:1087800000910905007809F011E3199304E00C94B5
:108790005F3A0E94DC48023012F00C94453AF8949B
:1087A000109109051F77002309F01068109309053F
:1087B000789404E00C945F3A112379F010E300916F
:1087C0003B0420913D04243024F400FD11E319936F
:1087D00014C007FD11E3199310C00E94DC48023059
:1087E00012F00C94453A112700FD10E1009154015C
:1087F0000F7E012B00935501789404E00C945F3AAE
:10880000112339F010E300911E0407FD11E31993C1
:108810000DC00E94DC48023014F00C94453AF894E4
:1088200006950795016000931E04789404E00C946B
:108830005F3A112331F133270091A7021091A8026A
:10884000112381F41091170100911801055C10406B
:1088500032F400E30993099305E00C945F3A21E4B4
:108860000E94BF49222711275FEF48E00E9445324E
:108870000091DA0109930091DB01099305E00C9462
:108880005F3A62E00E94A54812F40C94453A1D300C
:1088900010F00C94453A1093A7020FEF0093A80232
:1088A00005E00C945F3A112351F010E30091FF04AE
:1088B00006700695010F099304E00C945F3A0E943C
:1088C000DC48043012F00C94453AF8941091FF04FF
:1088D000197F000F102B1093FF04789404E00C9480
:1088E0005F3A112339F010E30091560105FD11E3C1
:1088F000199318C00E94DC4812F0023014F00C9456
:10890000453A10915601002319F415FF0BC002C01F
:1089100015FD08C0F8941091560100E2102710933D
:108920005701789404E00C945F3A112361F020E33E
:1089300000915401037019F000FD01C021E310E320
:10894000199329931FC00E94DC48002311F00C9456
:10895000453A0E94DC48023014F00C94453A32E06B
:10896000013041F00091540100FD0CC001FF0AC02C
:10897000332700C0F894009155010C7F032B00931E
:108980005501789405E00C945F3A442755276627F3
:1089900077271BC07091E6046091E7045091E804CA
:1089A0004091E9044A505040604070400EC07091C0
:1089B000E6046091E7045091E8044091E9048AE0FC
:1089C000480F80E0581F681F781F7093E60460937B
:1089D000E7045093E8044093E90403E00C945F3A01
:1089E000F6E1EBE905910993059109930591099346
:1089F00005910993059109930591099305910993AF
:108A00000AE00C945F3A112349F000919C024091D6
:108A10009E0240FD00919D020C944E3A63E00E943C
:108A2000A54812F40C94453A222311F00C94453ACF
:108A300010939D020FEF00939E0206E00C945F3AA4
:108A400000913005037011E4010F09930EE20993C0
:108A500000E3099300913005069506950395037090
:108A600010E3010F09930EE209930091300506957A
:108A70000695069506950F7010E30A3012F011E383
:108A80000A50199310E3010F09930AE00C945F3A1E
:108A90001123C9F100913F0409931091910301330F
:108AA000F1F0109195030233D1F010919403033348
:108AB000B1F010919603043391F0109198030533AF
:108AC00071F010919703063351F010919203073320
:108AD00031F010919303083311F00C94453A22279A
:108AE0005FEF48E00E9445320091D8010993009160
:108AF000D90109930091DA0109930091DB010993EF
:108B000008E00C945F3A0E94DC4812F0093014F03F
:108B10000C94453A006300933F0404E00C945F3AE0
:108B20000FEF00930B0503E00C945F3A112339F02B
:108B300010E30091EE0407FD11E3199318C00E94A1
:108B4000DC4812F0023014F00C94453A1091EE0417
:108B5000002319F417FF0BC002C017FD08C0F894DA
:108B60001091560108E0102710935701789404E003
:108B70000C945F3AF89400915A01086010E40E9446
:108B80000F3806ED0E945F3800270E945F38789406
:108B900003E00C945F3A112351F020E30E94F9386E
:108BA000007409F021E3299304E00C945F3A0E94D9
:108BB000DC48023012F00C94453AF894202F0E94C1
:108BC000F9380F7B222309F000640E93789404E0B7
:108BD0000C945F3AF89400915A01086010E40E94E6
:108BE0000F3806ED0E945F380FEF10913D041A30E8
:108BF00019F014300CF000E80E945F38789403E01C
:108C00000C945F3A112339F410E300912F0400FD16
:108C100011E318830BC00E94DC48023012F00C9460
:108C2000453A112700FD1FEF10932F0404E00C9428
:108C30005F3A112341F010E300910605010F0993FB
:108C400004E00C945F3A0E94DC48083012F00C9467
:108C5000453AF89400930605789404E00C945F3A42
:108C6000112381F0332722271127009105055FEF9B
:108C700048E00E9445320091DA0109930091DB013E
:108C800009930CC062E00E94A54812F40C94453A86
:108C9000153514F00C94453A1093050505E00C9435
:108CA0005F3A112381F03327222711270091040511
:108CB0005FEF48E00E9445320091DA01099300918C
:108CC000DB0109930CC062E00E94A54812F40C94E9
:108CD000453A153514F00C94453A1093040505E017
:108CE0000C945F3A112341F010E300910705010F46
:108CF000099304E00C945F3A0E94DC48053012F0BE
:108D00000C94453AF89400930705789404E00C9489
:108D10005F3A112341F010E300910305010F09931D
:108D200004E00C945F3A0E94DC48053012F00C9489
:108D3000453AF89400930305789404E00C945F3A64
:108D40001123C1F0332722270091B5021AE0019FB9
:108D500080015FEF48E00E9445320091D8010993FD
:108D60000091D90109930091DA0109930091DB0187
:108D7000099314C064E00E94A54812F40C94453A8B
:108D8000012F122F29E0073F120710F00C94453AEB
:108D900033272AE00E94BF490093FC0407E00C94AB
:108DA0005F3A112339F010E300913A0400FD11E31A
:108DB00019930BC00E94DC48023012F00C94453A23
:108DC000112700FD1FEF10933A0404E00C945F3A62
:108DD000F8941091DF040091E00478940754114056
:108DE00012F411270027332721E20E94BF491127DF
:108DF00000310CF00FE001952FE0020F22275FEF0A
:108E000048E00E9445320091D80109930091D901B0
:108E100009930091DA0109930091DB01099307E0BE
:108E20000C945F3A112349F0009185024091880229
:108E300040FD009187020C944E3A63E00E94A548E1
:108E400012F40C94453A222311F00C94453A1093F5
:108E500087020FEF0093880206E00C945F3A10E35C
:108E600000910A0501FD11E3199333272227109180
:108E70001B0100911C015FEF48E00E944532009108
:108E8000D80109930091D90109930091DA0109935E
:108E90000091DB01099308E00C945F3A0E94DC48E2
:108EA000023012F00C94453A10910A051B7F000F16
:108EB000000F102B10930A0504E00C945F3A33273F
:108EC000222710911D0100911E015FEF48E00E94D2
:108ED00045320091D80109930091D901099300917D
:108EE000DA0109930091DB01099307E00C945F3AE2
:108EF0000E94DC48023012F00C94453A10910A05A9
:108F00001E7F102B10930A0504E00C945F3A112386
:108F100029F00091FE0403950C944E3A63E00E9400
:108F2000A54812F40C94453A222311F00C94453ACA
:108F3000112311F01F3114F00C94453A1A95109337
:108F4000FE0406E00C945F3A112321F00091FA042C
:108F50000C944E3A63E00E94A54812F40C94453AF2
:108F6000222311F00C94453A112311F40C94453A44
:108F70001093FA0406E00C945F3A1123C1F03327F2
:108F800022271AE00091B402019F80015FEF48E0C0
:108F90000E9445320091D80109930091D9010993AB
:108FA0000091DA0109930091DB01099314C064E098
:108FB0000E94A54812F40C94453A012F122F29E083
:108FC000073F120710F00C94453A33272AE00E941D
:108FD000BF490093FB0407E00C945F3A112321F092
:108FE0000091B1020C944E3A63E00E94A5482223FE
:108FF00012F40C94453A1093F80406E00C945F3A8E
:10900000112389F00091010514E3002351F010E0D1
:10901000013039F012E3023021F011E3033009F09E
:1090200013E319931CC00E94DC48053012F00C9425
:10903000453A11E0002371F013E0013059F012E0DD
:10904000023041F014E0033029F01127043011F010
:109050000C94453A109301050FEF00934B0204E086
:109060000C945F3A112339F010E30091EE0400FDF7
:1090700011E3199318C00E94DC4812F0023014F07A
:109080000C94453A1091EE04002319F410FF0BC024
:1090900002C010FD08C0F8941091560104E010279A
:1090A00010935701789404E00C945F3A002711273D
:1090B000222733271BC03091EA042091EB04109142
:1090C000EC040091ED040A501040204030400EC0E6
:1090D0003091EA042091EB041091EC040091ED042E
:1090E0008AE0080F80E0181F281F381F3093EA0419
:1090F0002093EB041093EC040093ED0403E00C9434
:109100005F3A112381F0332722271127009113059D
:109110005FEF48E00E9445320091DA010993009127
:10912000DB0109930FC062E00E94A54812F40C9481
:10913000453A173114F00C94453A109313050FEF8C
:109140000093310405E00C945F3A1127222733275E
:10915000442755270D9109930E94D3480AF1100F17
:10916000251F351F451F6A95C9F0110F221F331F98
:10917000441F4F933F932F931F93110F221F331FB1
:10918000441F110F221F331F441F0F91100F0F9107
:10919000201F0F91301F0F91401FDCCF0027089533
:1091A0000FEF00230895005320F00A3010F400233D
:1091B00008950FEF002308950D910993005308952A
:1091C0000E94E838302F31702D911D910C915FEF86
:1091D00048E00E94453200E3099309930993009106
:1091E000D40109930091D50109930091D601099307
:1091F0000091D70109930091D80109930091D901F9
:1092000009930091DA0109930091DB0109930EE0C3
:109210000895712F0D9109930E94D3480AF42CC030
:109220000D9109930E94D3480AF426C00D91099329
:109230000E94D3480AF420C068E00E94A5480AF4BE
:109240001BC00C910B3309F017C04F933F932F9322
:109250001F93F894172F0E94E83811970E7F1F91E3
:109260002F913F914F91402B4D933D932D931C9304
:1092700078940EE0002308950FEF0023089510E086
:109280000E94E838402F4E701091FF0413FD409368
:109290003D041D912D913C91AF93BF930F931F936C
:1092A0002F933F9311E00E94E838402F4E70409377
:1092B0003C041D912D913C914F914C934F914E93B5
:1092C0004F914E934F914E93BF91AF913C932E93FC
:1092D0001E930E930895F89410E00E94E8380091D0
:1092E000DA060E930E7000933C041091FF0413FFF6
:1092F00000933D0411960091DB060D930091DC066E
:109300000D930091DD060D930091DE060D93009103
:10931000DF0600680C930FEF00930D040027009305
:109320007702009378020E94C73878940895A801C4
:109330005A014FE35527BA019A0185010E94BF499E
:10934000A8011A01260E371E36942794B101910107
:1093500085010E94BF49A8011A01260E371E3694C6
:109360002794B101910185010E94BF49A8011A010A
:10937000260E371E36942794B10181010895EE24FC
:10938000DD2480E1000F111FEE1CDD1CE216D30668
:1093900018F0E21AD30A03958A95A1F70895029F5F
:1093A000C001129F900D039F900D8C010895909124
:1093B000000597708827FAE1E0E65AE0589FD0014F
:1093C0005527A90FB51FEA0FFB1F35965491951726
:1093D00009F04CC0D0011496FAE1E0E6EA0FFB1F59
:1093E00054915E33B1F5FAE1E0E6E00DF11D7591BF
:1093F0006591559145910E94B538E4F1C1E04C2F3B
:10940000480F6AE0649FD0015527A90FB51FFAE104
:10941000E0E6EA0FFB1F359654919517B9F4D00199
:109420001496FAE1E0E6EA0FFB1F54915C3371F405
:10943000FAE1E0E6E00DF11D7591659155914591D8
:109440000E94B538CCF0C1F08C0F10C0C395C63067
:10945000B1F65D3359F4FAE1E0E6E00DF11D7591E6
:109460006591559145910E94B53831F083958732C9
:109470000CF4A1CF68940895E8940895B3E0A4EAA9
:1094800015E100E2F8940D931A95E9F700E20093D4
:10949000D3027894089520533AE0329F1053010E7E
:1094A0003327E4E3FAE10A95000FE00FF31F05917B
:1094B0001491000D131F0C5110402227552748E02E
:1094C0000E9445322091D9011091DA010091DB010F
:1094D00008950F7002951127B7E0A8E9A00FB11FFA
:1094E000F8E0EFE51CE022270D910C3309F42FEF93
:1094F000222309F000E201931A95B1F707E10093E6
:109500003704089510E00E94E8380E7011E3063029
:1095100099F012E3043081F013E3003069F014E3B2
:109520000A3051F015E3083039F016E30C3021F021
:1095300017E3023009F019E3089566E0013399F06A
:1095400064E0023381F060E0033369F06AE00433E1
:1095500051F068E0053339F06CE0063321F062E049
:10956000073309F06EE0089500EC00934804F89486
:109570000091640100640F7D10ED0E942B387894F7
:10958000F89400915D010170006D10E70E942B3886
:1095900000915A01086010E40E940F3806ED0E9405
:1095A0005F380FEF0E945F38789444E68DE07727AC
:1095B00066275527109166011078062F00950F77C2
:1095C000012B0E94CE4B10EF0E942B38052F0F77F6
:1095D000072B0E94CE4B10EE0E942B380E94B84BF6
:1095E0000AF48FC014E60091CB02023129F001E0A9
:1095F0000E94C74B1A95B9F74F935F938F930E94C0
:10960000E04B0E94FE4B0E94364C8F915F914F9130
:1096100000910201041738F45093EF066093EE06B0
:109620007093F006402F08170CF472C088945523ED
:1096300009F40894551F57FFBDCF8894662309F499
:109640000894661F67FFB5CF772311F470E8B0CF99
:1096500003E0800F89310CF4AACF8DE06091EE0613
:1096600066959091EE06992311F497E003C0990F47
:1096700097FD9FE75091EF0656953091EF06332303
:1096800011F437E003C0330F97FD9FE71091660197
:109690001078062F00950F77012B0E94CE4B10EF0C
:1096A0000E942B387091F006052F0F77072B0E9430
:1096B000CE4B10EE0E942B380E94B84B12F13F9314
:1096C0004F935F938F939F930E94E04B0E94FE4BBA
:1096D0000E94364C9F918F915F914F913F910091E5
:1096E0000201041728F45093EF066093EE06402F12
:1096F000081774F05395531749F66395691709F0E5
:10970000B9CF0FE70093EC0600270093ED0612C0D7
:109710000091EE060E94CE4B00950F770093EC0669
:109720000091EF060E94CE4B0F771091F006012BAF
:109730000093ED06F89400915A01086010E40E942D
:109740000F3806ED0E945F3800270E945F380091B5
:109750005D0110E70E942B380091640110ED0E941A
:109760002B38009148040F7B0093480478940895A7
:109770000BE0009343040091540105FD02C02894BE
:109780000895009143040023B1F7A894089500932D
:109790004304009143040023E1F70895102F10784B
:1097A00000FD106401FD106202FD106103FD1860F0
:1097B00004FD146005FD126006FD1160012F08957F
:1097C000F894B1E0A6E30027112748E03D912D91E0
:1097D000020F131F4A95D1F77894169507951695A1
:1097E0000795169507950E941C4CF89430939303A7
:1097F000109305010093060178940895F894B1E060
:10980000A6E20027112748E078943D912D91020FA0
:10981000131F4A95D1F71695079516950795169536
:1098200007950E941C4CF894309392031093030107
:109830000093040178940895169507951695079559
:10984000009F112D2EE2129E110E1F922BE6129FE9
:1098500080012091FF042670243031F0263021F061
:109860002AE033270E94BF493F9108957894112739
:10987000009192031093480100934901000F111FBA
:10988000000F111F000F111F000F111F000F111FDC
:10989000000F111F0E9497491F930F9311270091EA
:1098A000930310934A0100934B01000F111F000F07
:1098B000111F000F111F000F111F000F111F000FAC
:1098C000111F0E94974930914801209149010E943F
:1098D000CF49000F111F2F913F910E94BF49309136
:1098E000480120914901020F131F30914A01209134
:1098F0004B01A901020F131F2AE033270E94CF4911
:109900003091480120914901241B350B1AF00901BF
:10991000102811F4332721E00E94BF490F931F93B1
:109920001AE0019FF89400920201109201017894CC
:109930001F910F910A50104010F400271127102F8B
:10994000002728E233270E94BF490093910308951E
:10995000B1E0A0E0F8E0EBEBF8940C9111270E9445
:10996000CF4CB1F41FEF0E94CF4C91F41AEA0E9441
:10997000CF4C71F415E50E94CF4C51F40C93119625
:10998000AE17BF0749F778940AE100937F02089564
:109990000C9378940AE1019500937F0208951C933B
:1099A0002C9112170895309146073323E1F7D7E041
:1099B000C8E430E239933327222711275FEF48E0CC
:1099C0000E9445320091D90109930091DA0109936F
:1099D0000091DB01099305E00E945F3A0895599ACE
:1099E0000E942E350E942E350E942E350E942E3563
:1099F0000E942E355998089520913D04243029F075
:0C9A0000263019F02C3009F02E300895AB
:00000001FF
